:020000020000FC
:02000000EEC050
:02000800567828
:100034000C94662F0C94642F4156522D43686970BA
:100044004261736963322028632920323030362DAF
:1000540032303039204A6F65726720576F6C667290
:04006400616D0000CA
:10007000C8EDD1E00895C4E1D1E00895C0E0D1E039
:100080000895CCE3DDE00895E0E0F6EF0895E0E0C8
:10009000F6EF0895FF91EF91EF93FF93EF2FE85460
:1000A000F2E4FA5FE650E8F7EE270895009338018E
:1000B000089500913801089500934A010895009130
:1000C0004A01089500931B0108950C94EA360C949C
:1000D000A8320C941B330C9438320C9493320C9449
:1000E000C6340C94A5340C94AD340C94D7350C94D0
:1000F0001C3D0C94E8320C9413370C941A37409141
:10010000200108954091220108954091230108950E
:100110004091210108950C948F380C949B380C94D5
:10012000AB380C949B370C94CB3D0C94A83D0C94AD
:10013000D9340C94B5360C94F6350C940F360C94D7
:10014000263B0C946D3B0C94D2390C94B2390C9430
:10015000C3390C94C2380C9415390C94B03B0C94F0
:10016000D93B0C94A33B0C94CC3B0C94F3360C94ED
:100170001E3E0C94313E0C94EC3D0C94E83D0C94E6
:10018000F23D0C94F73D0C94EE3D0C943C3E0C94E7
:100190005E3E0C94673E0C947D3E0C94843E0C9421
:1001A000D63F0C94BA400C942D410C94A3410C946E
:1001B00049410C945D400C94A43E0C94B23E0C94C6
:1001C0003C400E9425410C94FB3E0E94C73E0C948B
:1001D000B73F0E94813F0C94E33E0C94293FF89472
:1001E000A0E02A2EA1E03A2EA0E1AEBFAFEFADBF56
:1001F0000E9427310E94E13D0E9416790E94283911
:100200000E94A832AFEFA0931001A0933D0120926D
:10021000490120924A0120925C018827789420921B
:100220003901A0913501A4FD0C942F010E94A83240
:100230000E9404040E941337D2CFAF91BF91CF9197
:10024000DF91EF91FF9108950F901F90FF93EF932F
:10025000DF93CF93BF93AF931F920F920895A1E0C6
:100260000E941532AA270E94A1319927A7E10E9476
:1002700010320E94A832A0E10E941032C4E0DAE0FD
:10028000E7E3F7E10E940F36A7E00E9410320E94D8
:10029000AD340704200030D1A6E10E941032C5E041
:1002A000D8E0E6E0F9E00E940F36D8E1F9E10E94DB
:1002B0000F36D8E0F9E0CC5FEC5FC833A0F368E715
:1002C0000E94EA364091200141FD0EC06A95C1F7B7
:1002D00056E142E00E941C3D0E94EA360E94EA3646
:1002E0005A95B9F70C9491010E94A8320E94AD343E
:1002F00000004B6579626F6172642D546573740000
:100300000E94E83270918101A0918101A215E1F370
:100310002092810190E07A2F0E9493320E941A333A
:10032000F3CFA0E00E941532A1E00E947A3899270D
:1003300020923601AA270E94A131A5E10E94103225
:100340000E94A832C0E0D0E0EDE1F4E10E94523614
:10035000A1E50E9410320E94AD34010183838383A2
:100360008383204156522D436869704261736963EB
:1003700032208282828282820000A9EAB4E00AE40A
:100380000D9304EC0D930CE80D9308E20D9302E637
:100390000D9306EA0D93509606EA0D9302E60D932F
:1003A00008E20D930CE80D9304EC0D930AE40D9311
:1003B00081D2409149014B3008F0442740934901D4
:1003C000642F67FD66276B3008F06AE050E06F939A
:1003D000A6D06F9153955830D1F761D136D10BD15A
:1003E0006F9387D16F91423E11F46A95EACF433EF5
:1003F00011F46395E6CF443E21F4643010F064506C
:10040000E0CF453E21F4673010F46C5FDACF6830FE
:10041000F8F04A3E11F0443F19F760934901683003
:1004200039F44A3EE9F676D00E94141E73D079CF93
:10043000693039F44A3EA1F66DD00E94D7226AD0C5
:1004400070CF68D04A3E61F60E94C02463D069CF65
:100450004F934091200142FD2AC04F914A3E11F036
:10046000443F41F46093490155D088270E94040419
:1004700051D057CF413F41F4609349014BD0882779
:100480000E94EA0347D04DCF423F39F460934901BF
:1004900041D00E94C21F3ED044CF433F39F4609305
:1004A000490138D00E94292035D03BCF99CF4F91B8
:1004B000413F39F4609349012DD00E948F032AD027
:1004C00030CF423F39F46093490124D00E94642523
:1004D00021D027CF433F39F4609349011BD00E94BC
:1004E0009F2518D01ECF443F09F76093490112D0D1
:1004F0000E94D7030FD015CF0E94AD34FF41565252
:100500002D436869704261736963322056302E3919
:1005100034000895A0912201A030E1F70895A1E0F0
:10052000B3E050FDA95F51FDA25F52FDBA5F452FB8
:100530000E94B579042F4EE20E3409F44CE265179F
:1005400009F44295409338010E94C6340E94AD34AC
:10055000FF20200040E50E941B33452F4F5C0E9486
:100560001B330E94AD34FF202000B3950E94C63497
:10057000452F0E94B5794E3481F40E94AD34FF209E
:1005800020E6E7202000B3950E94C6340E94AD34D7
:10059000FF2020E8E92020000FC00E94AD34FF209A
:1005A00020D0D1202000B3950E94C6340E94AD34E3
:1005B000FF2020D2D3202000452F0E94277AB39518
:1005C0000E94C63466E045910E941B336A95D9F7B4
:1005D000B3950E94C63466E045910E941B336A952C
:1005E000D9F7B3950E94C6340E94AD34FF20202075
:1005F0002020200008954AE26A3009F44295409391
:1006000038010E94AD340F0F202020202020000050
:100610000E94AD34100F2020D4D5202000000E946D
:10062000AD34110F2020D6D7202000000E94AD3419
:10063000120F20494E464F2000000E94AD34130F88
:100640002020202020200000089548E2693009F48D
:100650004295409338010E94AD340F08202020209D
:10066000202000000E94AD3410082020D8D920207E
:1006700000000E94AD3411082020DADB20200000A9
:100680000E94AD341208434F4E46494700000E9475
:10069000AD341308202020202020000008954CE2D3
:1006A000683009F44295409338010E94AD340F013F
:1006B00020202020202000000E94AD3410012020A6
:1006C000DCDD202000000E94AD3411012020DEDF9F
:1006D000202000000E94AD34120144464C41534892
:1006E00000000E94AD3413012020202020200000B3
:1006F00008953DED209223010E94C03740912001D2
:100700004470431739F0342F403011F4D3D0F4CF74
:10071000ECD0F2CF40912301403071F30895A4E072
:100720000E941032C1E0DFE0ECE1F3E10E945236BA
:10073000A0E40E9410320E94AD341002436F707921
:100740002050726F6772616D20746F007091490163
:1007500060E0ACE0671709F4A0E60E941032B2E155
:10076000A62FAA0FA60FAD5F0E94C63440E50E94D7
:100770001B33462F47704F5C0E941B3363956830D4
:1007800041F70E941337423E21F47030D1F37A953D
:10079000DFCF433E21F47730A1F37395D9CF4A3EA2
:1007A00019F40E945A7A08954D3E59F708950E940F
:1007B000CC3B4F436C656172207468697320507242
:1007C0006F6772616D3F2000413009F008950E940B
:1007D000347A0895A0912201A030E1F70E94B37904
:1007E0004E3441F00E94F90420923901A091230176
:1007F000A43F09F096CD08D00E941A37A0E00E94CD
:10080000A1310E94A832E6CF0E94A8328827209208
:1008100022010E94257A3C9645914E3429F4339664
:10082000F695E79509957DCD0E94780E20921901E5
:1008300020925C01209236010E94E832A7E20E94D9
:10084000103292E0A0914A01A03079F0A33021F457
:10085000A7E20E94103209C0A0E10E941032A0E479
:10086000A0930001A0EEA0930101B6E1A0914A017E
:10087000A03079F0B9E6A13061F0B2E4A23049F0DD
:10088000BFE2A33031F0B8E3A53019F0B1E0A630F3
:1008900060F0AA270E94C6340E94AD34FF20505257
:1008A00045535320455343200000A0912201AD3E03
:1008B000E1F70895A0E00E9410320E94AD341500C7
:1008C0002020202020202020202020202020202028
:1008D0002020202020202020202020202020000058
:1008E000E4EFF8E00E9415390895E2E1F9E00E9492
:1008F0001539089520202020202020456469742087
:10090000205361766520204C6F6164202052756E03
:10091000202020202020202020436F707920205389
:10092000656E642020526563762020436C65617299
:10093000AA270E941532A3E00E947A388F93409133
:1009400049010E9421790E94A8320E94963199277C
:10095000409122014030E1F70E94AD340000205068
:10096000524F4752414D2000409149014F5C0E9437
:100970001B334AE30E941B33C3EED1E058D2F0D2BE
:100980000E94F479EBD38F91A8E8803069F1ACEC48
:10099000E6E9F1E1813031F0ABE48A9545914030F0
:1009A000E9F7F8CF4CD292E0A5E0B1E00E94C6345E
:1009B0000E94A5340E94AD34FF20494E2050000013
:1009C000409146014F5C0E941B334AE30E941B3357
:1009D000BB27AC2DA3950E9438324AE30E941B33FB
:1009E000AD2DA3950E9438320895AAE25A2E70E2E6
:1009F00008959927FADF9CDFD22CAA27BB27D09233
:100A00003A010E943D370E94C037403E11F4AA27A8
:100A1000F6CF413E11F4AFE12BC0423E11F4AA954E
:100A200027C0433E69F4A3959B2F0E94070A9A179B
:100A300030F4BE3511F4AA951BC0AA27B39518C08F
:100A4000443E21F4BA95B7FDBB2712C0463E21F4BF
:100A5000B850B7FDBB270CC0473E11F4B85F08C0C3
:100A6000453E11F4B39504C04A3E39F5B395AA2723
:100A7000A03838F0AFE1BA95B038C0F0AA27BB274C
:100A8000BECFA03228F0BE3589F0AA27B395B7CFE4
:100A9000BF3508F0BEE50B2F0D1508F4D02E0D2D37
:100AA000015F0B1718F40B2F0F50D02E9B2F0E94B5
:100AB000070A9A1708F4A92FA2CF9B2F4E3E39F4AC
:100AC000AF93BF930E94C909BF91AF9189C14F3EB7
:100AD00031F4BF930E94D409BF91AA2781C1493E36
:100AE00011F482D17DC14C3E31F4A03009F489CF9C
:100AF000AA957AD175C150912001547009F4C5C0EE
:100B0000433FD1F4ACEC9BD10E94AD340107524578
:100B100043454956452050524F4752414D20592F89
:100B20004E203F006DD12EF475D218D35EDF509267
:100B3000D8017DD1882761CF423F39F5ACEC7FD118
:100B40000E94AD34010753454E442050524F475246
:100B5000414D20592F4E203F000052D156F7ACECAA
:100B60006ED10E94AD34010753454E44494E472E85
:100B70002E2E202020202020202000003092360120
:100B800093D12092360131DFD4CF443FB1F4ACECA5
:100B900056D10E94AD340107434C4541522050527A
:100BA0004F4752414D20592F4E203F0029D126F466
:100BB000C3D21BDF5092D801BCCF413F41F5ACEC12
:100BC0003ED10E94AD3401075052494E542050523C
:100BD0004F4752414D20592F4E203F0011D1B6F4BE
:100BE000ABE42DD10E94AD3401075052494E544917
:100BF0004E472E2E2E202020202020202000A2E054
:100C0000A093360151D120923601EFDE92CF4336C8
:100C100071F462E46093F50165E56093F60166E4C2
:100C20006093F7016DE36093F80161D2EACE483733
:100C300091F462E46093F50165E56093F60166E482
:100C40006093F7016DE36093F8010E94770864D226
:100C50005092D80118C04637B1F46091F501623462
:100C600099F460E26093F5016093F6016093F701F7
:100C70006093F8016093F9016093FA012BD26ED270
:100C80005092D801BECE8827BCCE423F11F5BF930B
:100C9000AF93C9D0D9F0ACECD2D00E94AD340107EB
:100CA000534156452050524F4752414D20592F4EE7
:100CB000203F0000A5D046F40E94C0790E94F4793C
:100CC0004DD293DE7093D801B2D08827AF91BF91F7
:100CD00096CE433FE1F4BF93AF93A5D0B9F0ACEC0F
:100CE000AED00E94AD3401074C4F535420434841CD
:100CF0004E47455320592F4E203F000081D026F704
:100D00000E94F4792BD271DE7093D801DDCF413F80
:100D100049F46A2E7B2EADD0A62DB72D5092D80166
:100D200070CED2CF4D3E09F5BF93AF937CD0A9F0E2
:100D3000ACEC85D00E94AD34010751554954205781
:100D40002F4F205341564520592F4E203F0058D059
:100D500046F7A0912201A030E1F70E948E31A0E079
:100D60000E94A131AF91BF910895443FE1F45BD05F
:100D700029F40E948E310E94A8320895A9E65FD01E
:100D80000E94AD34010753415645204348414E4728
:100D90004553204245464F52452052554E210000B2
:100DA0000E94133791CF5091200152FD1CC053FD7A
:100DB0001AC04C31C0F04038B0F4AF3171F05A2F46
:100DC000AFE10E9492376A916983AA95A517D9F776
:100DD0004883A3955092D80114CE0E94923748833D
:100DE0005092D8010ECE0DCE0E9492375A2F5F310D
:100DF00021F0498149935395FACF50E258830895E1
:100E00000E941337493559F0493749F04A3E39F0C5
:100E10004E3439F04E3629F04D3E19F0F1CF68943A
:100E20000895E8940895A091D801A0320895A8E803
:100E300006D00E94AD3401054F4B00000895EF939A
:100E4000FF939927A0934C010E94AD340105202007
:100E50002020202020202020202020202020202092
:100E6000202020202020202020202000FF91EF9112
:100E70000895A0E00E9465374A3E09F40895423E75
:100E800021F4A030B9F3AA95F5CF433E21F4AB305D
:100E900089F3A395EFCF403268F3403858F7488381
:100EA000AB3009F0A395E6CFC9EDD1E056E1499109
:100EB0000E941B335A95D9F70E94E8324EE511D0B3
:100EC00016F04A95E1F7542F53954427451719F02A
:100ED00024D04395FBCF43E20E941B330E94E832AB
:100EE0000895CF93DF935F936F93E894C4E4D2E0C7
:100EF00053E2459FC00DD11D50E26991613238F433
:100F00005A95D9F76F915F91DF91CF9108956894C9
:100F10006F915F91DF91CF910895DF93CF934F93BE
:100F20005F936F93C1E4D2E053E2459FC00DD11DA2
:100F3000DF93CF93A39653E26A91613210F45A95EE
:100F4000D9F7CF91DF9149910E941B335A95D9F778
:100F50000E94E8326F915F914F91CF91DF91089598
:100F6000AF93BF93EF93FF934F93E8E8FFE0AEE1B9
:100F7000B2E04591403011F04D93FBCF4F91FF917E
:100F8000EF91BF91AF91089520457869742020209A
:100F90004E616D6520202053617665202052656C7E
:100FA0006F616420202052756E202000AF93BF93A4
:100FB000EF93FF934F93ECEBFFE0D9CF202020205D
:100FC000202020205072696E74202053656E6420AA
:100FD000202052656376202020204E657720200057
:100FE000AF93BF93EF93FF934F93E0EFFFE0BFCF3B
:100FF0002041626F72742020202020202020202099
:1010000020202020202020202020202020202020E0
:1010100020202000E5DFACEC12DF0E94AD3401059A
:10102000524543454956494E472E2E2E00002092E8
:101030003A010E949C089927ECECE0934C01E3EE06
:10104000F1E0EE2EFF2E41E10E948F385CE00E941D
:10105000AB384B31B9F14A33D1F70E94AB384B3141
:1010600089F1403218F041935A95B9F7403228F08F
:101070000E94AB384B3131F1F9CFEEE1F2E0EE2EC8
:10108000FF2E53E2EE2DFF2DB396EE2EFF2E0E9483
:10109000AB384B31B9F04032D0F3433299F006C04F
:1010A0000E94AB384B3171F0403248F041935A9571
:1010B000B9F70E94AB384B3129F04032D0F7939505
:1010C0009036F9F60895A3E2BA9FA1E4B2E0A00D2C
:1010D000B11D0895BF93AF93F6DFC8E8D1E053E2A6
:1010E00049914D935A95E1F7AF91BF910895BF9300
:1010F000AF93E9DFC8E8D1E053E24D9149935A95A7
:10110000E1F7409188014093F901409189014093B2
:10111000FA01AF91BF910895BF93AF934F935F933F
:10112000D2DF139640E250E24D935A95E9F75F9172
:101130004F91AF91BF910895DF93CF93BF93AF933A
:101140004F9340E2A1E4B2E0CDEFDCE04D93219774
:10115000E9F74F91AF91BF91CF91DF91DF93CF939B
:10116000BF93AF934F9341E0A1E4B2E0C0E3D42F2B
:10117000DA5010F0C395FCCFD65CCD93DD93C0E27E
:10118000CD9390964395403689F74F91AF91BF919B
:10119000CF91DF910895425245414B004F56455241
:1011A000464C4F5700444956494445202F30005380
:1011B00051522046524F4D203C3000434F4E535425
:1011C000414E5420544F4F204249470057524F4EF2
:1011D000472045585052455353494F4E0053594E9E
:1011E000544158204552524F5200554E4B4E4F5786
:1011F0004E204B4559574F52440057524F4E4720AF
:10120000464F524D415400424144204C494E454EB8
:10121000554D424552004E45585420572F4F2046B9
:101220004F520052455455524E20572F4F20474F92
:1012300053554200544F4F204D414E5920474F5374
:10124000554200544F4F204D414E5920464F5200B9
:10125000493243204552524F5200554E4B4E4F5744
:101260004E204552524F520044464C41534820456F
:1012700052524F52004F5554204F46204152524136
:101280005900494E434F4D504C4554452050415212
:10129000004B4559574F5244204953204D49535311
:1012A000494E470057524F4E472042434F50592016
:1012B000004F5554204F462053435245454E00435E
:1012C000414E4E4F54204352454154452046494CCF
:1012D00045004D454D4F52592046554C4C0046490E
:1012E0004C45204E4F5420464F554E4400504147E8
:1012F00045204E4F5420494E2046494C4500504110
:10130000474553204E4F5420494E2052414E4745A9
:10131000004E4F5420494E204752415048494353B4
:10132000204D4F4445004E4F5420494E20544558BF
:1013300054204D4F4445004E4F20555352204649AE
:101340004C4500535243204F5554204F46205343A1
:101350005245454E0044455354204F5554204F4666
:101360002053435245454E0057524F4E472053504D
:10137000524954450057524F4E4720454550524F11
:101380004D20414452004E4F205052472046494C78
:101390004500BE3508F00895BF9328D0B395BE35FB
:1013A000E1F7BADEBF91DACEBE3508F00895BF93FB
:1013B000AF93AB2FAA95BDE508D0BA95BA17E1F760
:1013C000B395AADEAF91BF91C9CEBF93AF93DF9320
:1013D000CF9379DE1396ED01B0E2A991AAA3BA9555
:1013E000E1F7CF91DF91AF91BF910895BF93AF9394
:1013F000DF93CF9368DE1396ED01B0E2ABA1A99322
:10140000BA95E1F7CF91DF91AF91BF910895BF9366
:10141000AF93DF93CF9357DEED0193964E91413218
:10142000E8F34038D8F7AC1BBC0B9A2F925097FDCD
:101430009927CF91DF91AF91BF910895CAEFDCE07A
:101440002A922A9280E02F92AA27BB2744277191E3
:101450007032E9F37C3121F4A191BB27719126C050
:101460007E3121F4A191BB27719120C07D3121F4FF
:10147000B191A19171911AC07F3121F4B191A191E3
:10148000719114C07C3130F4572F4C2E5D2ECE2F2D
:10149000DF2F1AC0703398F07A3388F4403810F098
:1014A00086E0FAC0A72FA053BB2771914F3709F4EC
:1014B00059D1AA93BA9340E8CDCF85E0EDC07134FD
:1014C00000F17B35F0F40BC05F93452FAA27BB27B3
:1014D000EC2FFD2FC42DD52DBACF87E0DDC04038CD
:1014E00010F086E0D9C07154770FEF93FF93E0EAD4
:1014F000FCE0E70FF21DA191B191FF91EF91719185
:10150000D5CF7D3251F44F3711F44427A0CF20F4CA
:10151000403210F04FE79BCF78C0783231F471E061
:101520007F93AA27BB27472F92CF793209F067C054
:101530005F91513019F0523011F40CD15CC053302E
:1015400011F41CD158C0543029F4D5D1803009F0A1
:10155000A3C04FC0553029F4B991A991B095A09579
:1015600048C0563009F4DEC1573009F48EC25830F5
:1015700009F4C8C2593009F4DDC25A3009F4F9C27D
:101580005B3009F401C35C3009F402C35D3009F437
:1015900004C35E3009F4DAC2503109F40BC2513190
:1015A00009F42EC1523109F431C1533109F40FC28B
:1015B000543109F424C25F3009F440C3553109F4B1
:1015C000BDC1563109F4D1C1573109F4D6C15831E2
:1015D00009F46FC2593109F482C25A3109F440C387
:1015E000503029F06ED0803009F056C0A1CF86E08F
:1015F0000895AA93BA93AA27BB2742E028CF4F3772
:1016000020F44F3010F086E047C07C3361F471E283
:1016100060816E3319F472E2619142C06D3311F44E
:1016200073E261913DC07E3339F474E260816D33C1
:1016300011F475E2619134C07D3311F476E230C06B
:101640007B3211F470E32CC07D3211F471E328C0B9
:10165000733211F472E324C07A3211F470E420C0C2
:101660007F3211F471E41CC0753211F472E418C0B9
:10167000763211F473E414C05F91503021F05F3181
:1016800030F01FD0F9CFB991A9913197089586E034
:101690005F915030C1F3FCCF4F914030E9F708958E
:1016A0005F91A72FB52FA07FB07FBA1720F009D088
:1016B000803091F7F5CF5F937F93AA27BB27472F01
:1016C000C6CE5F934F9319910991B991A991513267
:1016D00011F4FED03AC0523221F4F3D0A150A170DF
:1016E00034C0533221F4FCD0A150A1702EC054322A
:1016F00011F4F6D02AC0553221F4EAD0A150A170DD
:1017000024C0563211F4DDD020C0503311F441D042
:101710001CC0513311F43CD018C0523319F4A02B23
:10172000B12B13C0503411F43FD00FC0513411F419
:10173000A7D00BC0523421F4A3D0A22FB32F05C0E1
:10174000533419F4A023B12300C0AA93BA934F9144
:101750005F910895B991A99103D0AA93BA9308957E
:10176000B7FF0895A095B095A30DB21D089517FF7A
:10177000089500951095030D121D0895B991A99132
:10178000AB2B29F0B7FBA1E0BB270EF41297E5CFF6
:10179000F0DF2B2F2127A00FB11F27FD08952B2F3E
:1017A000212727FD82E008950CD0A22FB32FBF7709
:1017B0000EF4D8DF37FD03C0452B09F4089582E00D
:1017C00008957AD0CDDFB19F402D512DA09F202DBF
:1017D000312DA19F300D411D521DB09F300D411D77
:1017E000521D089508E611E0B03818F0A00FB11F9F
:1017F000FBCFA017B10718F0A01BB10BFACF0895CB
:10180000B991A9910AE5A01BB20902C0B991A991A9
:10181000E9DFFF93EF93E6ECF3E80AE510E0A017A9
:10182000B10748F4E00FF11FEA1BFB0BA491EF9105
:10183000FF91BB27DECE04EB10E0A017B10778F4D0
:101840000AE510E0E01BF10BEA0FFB1FA491EF91FA
:10185000FF91BB27A095B095A30DB21DCACE0EE097
:1018600011E0A017B10728F4E00FF11FEA1BFB0BF2
:10187000EDCF0EE011E0E01BF10BEA0FFB1FD6CF1E
:10188000212F202B11F483E0089516D0222733272F
:10189000442751E1441FAA1FBB1F5A9551F0221F34
:1018A000331F4FEF201B310BA8F7200F311F40E0F3
:1018B000F1CF0EF457CF08952B2F212727FB50DFB0
:1018C00056CF0A271B27AA27BB27012B89F008958B
:1018D000B0581058A01BB10BAA27BB2748F0089599
:1018E000B05810580A1B1B0BAA27BB2708F00895F5
:1018F000A1E0B0E00895B991A99184E0B7FD089501
:1019000088270A2F1B2FB2E0AA27232D3327021B7B
:10191000130B20F0A3952B0F321DF9CFBB27AA93F1
:10192000BA9308954F935F930E94373919910991A3
:101930004ADFA42FB52F5F914F915BCE199109918A
:10194000023039F420925C01A2E0A0933F01BB2752
:1019500050CE013031F4A0913F01A03011F430920B
:101960003F01A0913F01BB2744CE199109910EBDC3
:101970000E94141AAEB5BB273CCE10914A0110301C
:1019800011F08CE1089519910991A4ECB2E00A17C5
:101990001B0710F082E10895FF93EF93FDE0ECE365
:1019A000E00FF11F68940E94C238EF91FF91A42FBD
:1019B000BB271FCEB991B0938301A991A093820157
:1019C000CF93DF930E94201ADF91CF9112CEB9916D
:1019D000A991BF3F71F0A09368010E94B7228030A7
:1019E00021F0AFEFBFEF882704CEA42FBB270C94C4
:1019F000F90A0E94BC228827B42FAA27FACDB991F0
:101A0000A991BF3F21F5A0FD11C0DF93CF93FF93B4
:101A1000EF930E94B422803019F08827CC27DD276D
:101A2000DE01EF91FF91CF91DF91E3CDDF93CF9373
:101A3000FF93EF930E94B422803019F08827EE279D
:101A4000FF27DF01EF91FF91CF91DF91D2CDA093DE
:101A500068010E94B722803021F08827AA27BB277F
:101A6000C8CDDF93CF937F9377270E94BF22DF3FBC
:101A700041F4CF3F31F4A72FBB277F91CF91DF9166
:101A8000B8CD7395703889F7F6CFA991A991A77051
:101A9000A06CA0937C00A0917A00A064A0937A002F
:101AA000A0917A00A6FDFCCFA0917800B0917900BA
:101AB000A0CDB991A991BB3020F4BA3028F0A83C50
:101AC00018F0AFEFBFEF95CDEF93FF93E8EDF1E0A6
:101AD000EA0FFB1FA081BB27FF91EF918ACDB330A6
:101AE00018F4B23010F0A7FDD7CDDF93CF93CCE33D
:101AF000DDE0CA0FDB1F0E94A83DA62FBB27CF91B8
:101B0000DF9177CDB991A991B03061F4AF3F79F011
:101B1000A770A395B0B1B695AA95E9F7AA27AA1F11
:101B2000BB2767CDBA2FA0B1AB23BB2762CDA0B135
:101B3000BB275FCDB991A9917091650177700E9423
:101B40001E3E8030E9F4BB27A52F53CDB991A99152
:101B5000CF93DF93CA2FDB2F0E945E3EDF91CF91A0
:101B6000803019F4BB27A42F44CDAA27BB2782E2DB
:101B70008FCDA99179910E943C3E803009F439CDF6
:101B8000AA27BB278FE084CDB991A991BB2731CD7E
:101B9000B991A991AB2FBB272CCD0F93B991099186
:101BA000AA27BB27003019F4A091220145C00130BB
:101BB00029F4A0912201A030E1F33EC0023039F4B3
:101BC000A0912201A030E1F7A091230135C003309C
:101BD00019F4A091200130C0043039F400912001A3
:101BE00000FD119602FD119727C0053039F40091D0
:101BF000200101FD119603FD11971EC0063049F426
:101C000000912201023E09F41197033EA9F41196B6
:101C100013C0073049F400912201043E09F41196E3
:101C2000053E51F4119708C01F931091220101172E
:101C3000E1F71F91A02FBB270F91DBCCB991A991A0
:101C4000BB27A13021F4A0917D01A395D2CCA23075
:101C500021F4A0917E01A395CCCCA0917F01C9CCA9
:101C6000CF93DF93EF93FF936F927F924F930E94F6
:101C7000B23E4030A9F0342F3395ED010E94181A7E
:101C8000803071F521963E011A2F0027A02F0E9467
:101C900027410E94FB3E141721F003950317B1F76B
:101CA0001CC0E3010E94181A8030D1F4A03091F0DA
:101CB0002A2FA02F0E94CB41E3012196E8E8F1E012
:101CC0000E94181A803061F4B191AB1731F7219658
:101CD0002A95B1F7A02FBB2702C0AFEFBFEF88272F
:101CE0004F917F906F90FF91EF91DF91CF9181CCD9
:101CF000FCE0E0EAA0E0B4EBA193BA95E9F7F1E0EB
:101D0000E8E7B0E1A193BA95E9F7FDE0ECE3B0E0D4
:101D1000A193A193A193BA95D9F7DD24CC24209265
:101D20001B0120921901AEE0A0933801ACE3A0930F
:101D30005001AEE2A0935101AFEFA0938701A093B1
:101D40001001209213010E94A83220925C01A2E0AF
:101D5000A0933F01A6ECA0937A00409149014093E3
:101D60004601409343010E9421799C2D0E943179C4
:101D700021D0803039F4AC2DAF35B8F39CE02092FF
:101D80005C010895C0927D01D0927E0180937F0115
:101D9000813051F020925C01409187014F3520F451
:101DA000DD24C42E8827E1CF9CE020925C010895B9
:101DB000F7012AC0F1E0E0EB209236018827AD2D33
:101DC000BB27AB1709F171917F3FD1F07C31D1F086
:101DD0007E31C1F07D31A9F07F3199F0773281F009
:101DE000723241F471917F3F59F0773249F072328B
:101DF000C9F7E9CF7A3339F7B395AB1721F704C0A8
:101E00002FC071917191DFCF7091390170FF05C0C2
:101E100081E07E7F70933901089572FF11C0AB7F1E
:101E200070933901A0914A01A53011F0A03011F44E
:101E30000E94181DA0FF04C00F900F9081E008952C
:101E40000E94C03770911301703039F0A0911001D9
:101E5000DA94209213010C94EE1271917F3F19F4E1
:101E6000DD24C394089577FD2BC0703269F27A3374
:101E700011F4D394C9CF773219F27134D8F07B358D
:101E800028F070527134B0F07B35A0F4672E0E94B8
:101E900011187D3379F4D2DA803069F4762D7154DB
:101EA000770FDCE0C0EAC70FD21DA993B99381CFA9
:101EB000EF91FF9187E00895703810F487E078CFB4
:101EC0007F01E8E6F72FFF73EF0FFFE0F21D0994A3
:101ED00049C0F3C0D9C26CC13EC111C359C373C755
:101EE00064C369C36DC33AC0C0C6DEC66DC3D7C381
:101EF000F6C22CC45CC4B1C19EC4AEC4B3C422C279
:101F0000CEC2B8C4C3C4CAC487C583C107C1B0C2E6
:101F100064C10BC5CDC424C00CC52DC587C201C387
:101F2000F4C5E9C749C655C65AC6ACC1DCC62DC7FB
:101F3000BAC75BC66AC693C241C58CC658C1BAC28D
:101F4000CCC32EC3C6C4C8C476C1AEC16EC6CBC195
:101F500088E0089584E1089583E108950C94C718FA
:101F60000C94E1180E9415189CE0732C2092360105
:101F7000B191B032E9F3BA3321F0B73211F0BF3F7B
:101F800059F4319770FC0E94E83240913601443098
:101F900010F00E94E83D0DCFBB3311F47724E8CF59
:101FA000BC3291F440913601403031F40E941A3332
:101FB000BA2DB770D9F706C00E941A33B091370115
:101FC000B770D1F77724D4CF732CB332C9F42092F1
:101FD00068012092690132DA4A2F40933601443079
:101FE00018F4433001F4C4CF0E94EC3D683051F541
:101FF000509136015E7F0E94EE3D683119F5B8CFF1
:10200000B03411F5DDD740913601433018F40E9409
:10201000C634AECF39F4A0936801B0936901A093A0
:102020003701A6CF5FEF0E94EE3D683259F45A2F78
:102030000E94EE3D683231F45B2F0E94EE3D683223
:1020400009F496CF8FE00895B13229F4F7D99A2F89
:102050008FCF97CF8DCFB23241F441914F3FC9F32B
:102060004232C1F30E941B33F8CFB63291F4E6D965
:10207000B33010F082E10895CCE3DDE0CA0FDB1F3E
:102080004991403029F00E941B331196B330C0F3C0
:102090006FCFB53229F4D2D94A2F0E941B3368CFB3
:1020A0003197CCD9803009F00895903818F40E9407
:1020B00038325ECF0E9493325BCF703CB8F4A1E01F
:1020C00031D7B0914A01B63019F00E94A83270CED3
:1020D000A13029F00E94B2390E94C33969CEB09173
:1020E0006801B130C9F30E94B23962CEA2E01AD7BA
:1020F000A23081F5A0E8B2E060916801C0916A0168
:10210000D0916C01CA17DB0738F4ACE3BDE0CA0F0D
:10211000DB1F0E94CB3D4CCE82E10895A2E002D7A6
:10212000A030C1F0A13059F0A0916A01A770AA0FA8
:10213000B0913801B770A295BA2BB0933801A09135
:102140006801A770AA0FB0913801B07FBA2BB09385
:1021500038012ECE01CF703C10F00C94C819A3E0CA
:10216000E1D6A33018F1A0916801B0916901A09364
:102170008201B0938301A0916A01B0916B01A09399
:102180006801B0936901A0916C01B0916D01B0300C
:1021900011F4A03051F00D010E94201A0E946E1817
:1021A000D001803021F41197F2CF02CED5CE089520
:1021B000733C09F4FDCDA5E0B5D6A43068F0C5D7D1
:1021C0007F93EDD6E0937B01F0937C010E94F6357E
:1021D0007F9170933801ECCDBFCEA1E0A3D6A130A2
:1021E000D8F340916801417040931901E1CDA5E019
:1021F00099D6A43068F0A9D77F93D1D6E0937B011C
:10220000F0937C010E940F367F9170933801D0CDFE
:10221000A3CEA5E087D6A43068F097D77F93BFD62A
:10222000C0937B01D0937C010E94263B7F917093E9
:102230003801BECD91CEA5E075D6A43068F085D723
:102240007F93ADD6C0937B01D0937C010E946D3B00
:102250007F9170933801ACCD7FCEA3E063D6A230DE
:1022600080F073D77F93B0916801A0916A01A09329
:102270007B01B0937C010E94D9347F917093380127
:1022800097CD6ACEA5E04ED6A43068F05ED77F9396
:1022900086D6E0937B01F0937C010E94B5367F9156
:1022A0007093380185CD58CEA0914A01A03011F02D
:1022B0008CE10895A1E036D6A130A8F3A091680181
:1022C000B0916901CCE3DDE0CA0FDB1F409138011A
:1022D0004F93AF92BF920E94B03BBF90AF904F918F
:1022E0004093380165CDA0914A01A03011F08CE1F6
:1022F000089580D6C0938201D093830192D67C3218
:10230000F9F4A1E010D6A13070F2A0916801B0916B
:102310006901CCE3DDE0CA0FDB1F409138014F9328
:10232000AF92BF920E94D93BBF90AF90C091820103
:10233000D0918301499329924F914093380138CD30
:1023400087E036CDA0914A01A03011F08CE10895CC
:1023500051D6C0938201D093830163D67C3281F73A
:10236000A1E0E1D5A13009F0F7CDFF93EF93AF9253
:10237000BF92409138014F937F934F704093380143
:102380000E94DC1BC1E0D2E0ECE1F5E10E94523694
:10239000C0913801C295C09338010E94AD34030248
:1023A0000000A0916801B0916901CCE3DDE0CA0FA3
:1023B000DB1FA6E14991403230F0403820F40E9402
:1023C0001B33AA95B9F7772761E025D00E94FE1B41
:1023D000623079F4C0918201D0918301799329927E
:1023E0007F914F9140933801BF90AF90EF91FF9153
:1023F000DFCC7F914F9140933801BF90AF90EF9128
:10240000FF91C0918201D09183014FEF499349938D
:10241000CFCC87E0CDCC0E94B9188827603009F472
:1024200008950E946A20882762E00895A3E07AD583
:10243000A230A0F08AD67F93D0917C01C0917B011D
:10244000F0916801E0916A01E0937B01F0937C01D7
:102450000E94B5367F9170933801AACC7DCDA4E05F
:1024600061D5A43021F49BD50E94D735A1CC74CD81
:10247000A1E058D5A13090F0A0916801A295AA0FD3
:10248000AF7EA0931B0194CCA1E04CD5A13030F0DD
:10249000A0916801A150CA2EDD2408955DCDA1E070
:1024A00041D5A13030F0A0916801A150A0938701DF
:1024B0007FCC52CDA7E036D5A230D8F3C8E6D1E024
:1024C000E881EF70F1E0BA81B770BB0FB295B193BC
:1024D000EF702296AA95A130B1F76ACC3DCDA1E06C
:1024E00021D5A130D8F3A0916801A7700E94A13135
:1024F000A0914A01A73010F40E94A83259CCA1E063
:1025000011D5A13068F0A0916801B0916901B03097
:1025100019F4A03009F44CCC0E94EA361197F7CF99
:102520001BCD20925C01A2E0A0933F01A3E0FAD46E
:10253000A33058F1CCE3DDE0A0916801B0916901CE
:10254000B33020F5AC0FBD1FA0935E01A0936001D6
:10255000B0935F01B0936101AC1BBD0B00906A01A9
:102560000A94A00DB21DA00DB21DB33078F4AC0FCB
:10257000BD1FA0936201B0936301A0916C01A09371
:102580005C013092640120923F0112CC82E110CCB8
:10259000703C28F420925C01BF91BF910895BDC6A4
:1025A00046D5AB2B09F42CCC04CC703C10F00C9429
:1025B000E2193BD5FECBF70103D50E94C634F9CB17
:1025C00036D50E94F336F5CBA2E0ACD4A13019F099
:1025D000A23021F1C1CCA0916801AA95AF3510F0CD
:1025E0008AE0E6CBB0918001BB3010F08DE0E0CB0B
:1025F000AF93CCEFDCE0A5E0AB9FC00DD11DB39550
:10260000B0938001BD2DB395B068B993BC2DB9933B
:10261000B0914901B993DD24CF90089540916801AC
:102620004A950E94B5794E3469F4A0916A01B0913F
:102630006B01B630A8F6F695E795EA0FFB1F3896C2
:102640000995B6CBA0916A01AA95AF3548F6B0912D
:102650006801BA95B770B0934301B0918001BB3067
:1026600010F08DE0A5CBAF93CCEFDCE0A5E0AB9F05
:10267000C00DD11DB395B0938001BD2DB395B06849
:10268000B993BC2DB993B0914601B993DD24CF9095
:1026900040914301409346010E9421790895C5D499
:1026A000B0918001B03011F48CE00895BA95CCEF70
:1026B000DCE0A5E0AB9FC00DD11DB0938001B991C6
:1026C000B7FFF2CFBF77DB2EC99049914093460107
:1026D0000E942179089587E00895A7D4A2D4713487
:1026E000D0F37B35C0F77154770F672E9AD47D33C2
:1026F00091F70E941E0A803009F00895DCE0C0EADC
:10270000C60DD21DA993B9938CD4733C21F70E94B6
:102710001E0A4A2E5B2E803009F00895B091800188
:10272000BB3010F08EE00895CCEFDCE0A5E0AB9F6D
:10273000C00DD11DB395B0938001BD2DB395B99354
:10274000BC2DB99369924992599233CB6ED4B09112
:102750008001B03011F48BE00895BA95CCEFDCE045
:10276000A5E0AB9FC00DD11DB991B7FDF4CFBF77E8
:10277000B0937A0159907991BCE0A0EAA70FB21DFD
:102780000D911D91030D121D1E930E93A991B991E8
:1027900011960A1741F41B1731F4B0918001BA95D4
:1027A000B093800106CBC52CD0907A010895A091FA
:1027B0004A01A03011F08CE1089537D4BFEFB093F7
:1027C0008801B191B032E9F34B2FBF3F21F40E9451
:1027D000E8323197EECABA33D1F3BB3391F3BC324E
:1027E00031F40E941A33BA2DB770D9F7EACFB2325A
:1027F00041F441914F3F59F3423219F30E941B3388
:10280000F8CFB134B0F0BB35A0F4B154BB0FB093E6
:102810007A01B081B13418F0BB3508F40AC00AD48B
:10282000DCE0C0EA10917A01C10FD21DA993B993DF
:10283000C8CF87E00895FBD3803009F0BACA4A2F89
:102840004B2BE1F340912E014030E1F340912E01FA
:102850004030E1F71197F3CFEAD3A0932F01B09363
:102860003001EDCFC7D3A0912F01A993A0913001E2
:10287000A9939FCADCD34A2F0E948F38D3D37C32CE
:1028800021F4CFD30E941E0AF6CF93CA0E949B3830
:10289000A42FBB27AFD3A993B9938BCAF7019DD3BC
:1028A0004A2FD73020F4C03D10F40E94673E81CA01
:1028B000F70193D35A2FAC2FBD2F7091650177701C
:1028C0000E94313E0E94EA360E94EA360E94EA36B1
:1028D00070CAADD3A1B96DCAF7017FD3D030B1F4BE
:1028E000BC2FB770B39577276FE7A0FD70E8A0FD08
:1028F0006FEF77FB770F70F967FB660F60F9BA959A
:10290000C1F702B1072B062302B953CAD13041F4F3
:10291000B2B1C095BC23C095CA23BC2BB2B949CA79
:10292000D230E9F70E94021A44CA81D30E947A3851
:1029300040CA60D3C0938201D09383010991199159
:1029400010586FD37C32A9F448D3B058D058C01770
:10295000D10710F00C2F1D2FA017B10710F40A2F6C
:102960001B2FD0918301C0918201105809931993B4
:1029700020CA86E00895A0914A01A63029F0A370EC
:10298000A03011F08CE1089535D3C0938201D0932B
:10299000830147D37C3269F713D3C8EDD1E07EE1E0
:1029A0007B9FC00DD11DCA0FD21DBB27A881D0911E
:1029B0008301C0918201A993B993FBC9A0914A01F7
:1029C000A370A03011F08CE1089514D3C09382015C
:1029D000D093830126D37C3261F6F2D2C8EDD1E0E8
:1029E0007EE17B9FC00DD11DCA0FD21DA2EBCA0F85
:1029F000A2E0DA0FBB27A881A695BA2FA777B295D8
:102A0000B078AB2BBB27D0918301C0918201A993F1
:102A1000B993CFC986E00895EDD2C0938201D093D7
:102A20008301FFD27C32B1F7CBD2C8EDD1E07091F7
:102A30004A017770703021F5AF93BF93A695B69594
:102A40007EE17B9FC00DD11DCA0FD21D7881BF9141
:102A5000AF91A0FD7695B0FD7695B0FD7695A2EB91
:102A6000B2E0CA0FDB1FA88170FFA295A695A770E0
:102A7000BB27D0918301C0918201A993B99399C9D1
:102A80007130B9F4AF93A695A695A69575E17B9F95
:102A9000C00DD11DCA0FD21D7881AF91A2FD7295D4
:102AA000A1FD7695A1FD7695A0FD76957170A72F75
:102AB000DECF7230A1F4AF93A695A6957EE17B9F01
:102AC000C00DD11DCA0FD21D7881AF91A1FD7295A5
:102AD000A0FD7695A0FD76957370A72FC8CF7330B3
:102AE00071F4AF93A6957AE27B9FC00DD11DCA0FFA
:102AF000D21D7881AF91A0FF7295A72FB8CFAF9369
:102B0000A695A695A69570E1C2CFA0914A01A630E0
:102B100029F0A370A03011F08CE10895A3E002D257
:102B2000A33080F0A0916801B0916901B33010F03A
:102B300082E10895B23039F4A73F28F082E1089588
:102B400081E2089509CACCE3DDE0CA0FDB1FC09320
:102B50005201D0935501AC81A03091F3AE3180F792
:102B6000BB81B03069F3B73158F7C0916801D0919B
:102B700069012596BA9F000C111C000C111CC00D98
:102B8000C11DD330E8F6D0916A01C0916C01C093A9
:102B90005401D0935701CF3F51F0DF3F41F0CA0FAE
:102BA000CA95CE3138F4DB0FDA95D73118F40E948C
:102BB0004B3CFEC886E10895A0914A01A03011F077
:102BC0008CE1089532D2A0913901A460A09339011B
:102BD000F0C8A0913501A062A0933501EAC8A09188
:102BE0003501AF7DA0933501E4C8A3E09BD1A330AC
:102BF00009F0B2C90E94B722403310F08EE1089567
:102C00000E94CB228030D9F7D3C8A3E08BD1A33068
:102C100009F0A2C90E94B722403310F08EE1089556
:102C20000E94CE228030D9F7C3C8A3E07BD1A23066
:102C300019F0A33021F090C9A4E1A0936C010E9487
:102C4000C522803009F4B4C808950E94C82280309B
:102C500059F4AEC8A1E066D1A13009F07DC90E9447
:102C6000B722443191F38EE10895A2E05BD1A23006
:102C700009F072C9A0916801B091690140916A019F
:102C8000CCE3DDE0403041F0D395413029F0D395DD
:102C9000423011F082E108950E94C73E0E94B73F82
:102CA000803009F0089584C8A2E03CD1A23009F038
:102CB00053C9A0916801B091690140916A01CCE3C8
:102CC000DDE0403041F0D395413029F0D3954230DA
:102CD00011F082E108950E94813F0E94E33E80301E
:102CE00011F308954EC0F7014FD1A09384010E94C3
:102CF000EC3D6830B9F790FF28C0592F0E94EE3D97
:102D0000603481F7A030C9F0DDE0CCE3409184016C
:102D10004B0F4A1BC40FD21DA13039F00E94F23D67
:102D2000603579F55883AA95EFCF0E94F73D683555
:102D300041F558830E94E83D3CC80E94F23D503066
:102D4000A1F350938401A52FDFCF592F0E94EE3DB0
:102D50006831B9F43A2FDDE0CCE3409184014B0FA8
:102D60004A1BC40FD21D5881503011F4303031F05D
:102D70000E94EE3D683229F4AA9569F70E94E83D69
:102D800018C88FE00E94E83D089551D1A0936801D2
:102D9000B093690147D17C3249F4319642D1723205
:102DA00039F031970E941E0A99D1F4CF0C94D90EB4
:102DB0007191723231F07F3F21F0BB27A72F8ED166
:102DC000F7CF7081E7CFA0914A01A03011F48DE1D7
:102DD0000895A43011F0A63028F0A4D0A43079F4DE
:102DE0000C941519A7E09ED0B0916801B0935801DA
:102DF000B13039F0B23011F1B33009F43DC085E1A2
:102E00000895A730E1F7C8E6D1E0BA81B093550143
:102E1000BC81B0935201BE81B0935601B885B09386
:102E20005301BA85B0935701BC85B09354010E94F9
:102E3000D239803009F008950C94D80EA630F9F6F6
:102E4000C8E6D1E0BA81B0935501BC81B09352017C
:102E5000BE81B0935601B885B0935301BA85B09343
:102E60005401BB85B09357010E94D239803009F0DC
:102E700008950C94D80EC3CFA430E9F7C8E6D1E08A
:102E8000BA81B0935201BB81B0935501BC81B0931C
:102E90005701BE81B09354010E94D239803009F0AD
:102EA00008950C94D80EA0914A01A03011F08CE145
:102EB0000895F70192D0C0936801D09369015091B1
:102EC0008401A51708F45A2FA8E8B1E0503071F03A
:102ED0004D91A0938501B0938601A42FBB27FED00E
:102EE000A0918501B09186015A95F0CFAA27BB2702
:102EF000F5D00C94D90EA0914A01A03031F0A43045
:102F000021F0A63011F08CE10895A1E00BD0A130A2
:102F100040F0A09168014A2F43700E941C3D0C9420
:102F2000D80E1AC8F701A03009F40895DF93CF93A3
:102F3000C8E6D1E040E05A2F503029F4A42F7F0199
:102F4000CF91DF910895DF93CF934F935F930E94CA
:102F50001E0A5F914F91CF91DF91893121F488272B
:102F60007F01A42F0895A993B99343955A955030A2
:102F700019F371917032E9F37C3229F33197A42F60
:102F80007F01CF91DF910895A3E0CCDFA33009F555
:102F900090916801B0916A01A0916C010895D0915F
:102FA0006801C0916A01F0916C01E0916E01C093DB
:102FB0005201D0935501E0935301F09356010895C7
:102FC000A2E0B1DFA23029F4B0916801A0916A01BA
:102FD0000895AF91AF910C94AC0FA2E0A4DFA230A2
:102FE000C1F7C0916801D0916901A0916A01B091C7
:102FF0006B010895F70115D0713478F07B3538F402
:103000007154770FDCE0C0EAC70FD21D0895713606
:1030100020F07B3710F47156F4CF8F918F9187E0B9
:10302000089571917032E9F30895F7010895F70159
:103030000C941E0AEF93FF930E947F37EC2FFD2F15
:1030400000E00E941F3770913901713011F4872F11
:1030500009C04A3EE9F400938401003031F4AA2704
:10306000BB278827FF91EF910895C8E8D1E0A1918F
:10307000A9930A95E1F7AFEFA9930E944D1AE0EBEF
:10308000F1E00E941E0A8D010E943179D801E9CF3A
:103090004C3E49F40030A9F2AA940E947F37A0E286
:1030A000A8830A95CECF403228F24B3718F6AA2DC6
:1030B000AD3100F60E941B330395C3CF92E0BB27CE
:1030C000AC2DA3950E9438324AE30E941B33BB27E4
:1030D000AD2D0E9438320E941A330895DF93CF93AA
:1030E000BF93AF93A0916801B0916901B33098F498
:1030F000CCE3DDE0CA0FDB1FAF91BF91A883C09185
:103100006801D09169012196C0936801D09369014B
:10311000CF91DF910895B45090F0AA0FBB1FB33048
:1031200070F4CCE3DDE0CA0FDB1FAF91BF91A99330
:10313000B993C0916801D09169012196E5CF82E1F0
:10314000AF91BF91CF91DF91089570913801A0FFA9
:103150000895A33059F450916C015F70550F707F42
:10316000572B709138015093380108955091700198
:10317000F4CF0E94D122403011F466270895409385
:1031800070010E94C222413009F066270895A2E032
:10319000C9DEA130A0F0B1E0A13011F0B0916A0118
:1031A000A0916801A150A0931001B09311010E9459
:1031B000EA36B0931201209213010C94D80E0C94AD
:1031C000AC0FA3E0AFDEC0916801D09169014091DE
:1031D0006A0108EC1AE028ED31E0A23080F319F41E
:1031E0001CD00C94D80E60916C01F0916B01F170C1
:1031F000E0916A014CE3E40F4DE0F41F4427C40F53
:10320000D21D41910AD041914038C8F34058C40FB3
:10321000D21D6A9551F70C94D80EC017D10720F42F
:10322000DE01A20FB31F4C930895FF93EF930CE3BD
:1032300010E120EA3CE0B0916801B13019F5E8ED09
:10324000F1E0A0916A01B0916B01BF70AE0FBF1F9A
:10325000C0916C01D0916D01DF70CE0FDF1FE09146
:103260006E01F0916F01A217B30740F4C217D307A4
:1032700028F4319718F00D900992F5CFEF91FF9156
:103280000C94D80EB23009F5E8EDF1E0A0916A0196
:10329000B0916B01BF70AE0FBF1FECE3FDE0C091BA
:1032A0006C01D0916D01DF70CE0FDF1FE0916E01D8
:1032B000F0916F01A217B30708F7C017D107F0F616
:1032C0003197E0F20D900992F5CFB33011F5ECE3B0
:1032D000FDE0A0916A01B0916B01BF70AE0FBF1FFE
:1032E000E8EDF1E0C0916C01D0916D01DF70CE0F7F
:1032F000DF1FE0916E01F0916F01A017B10740F45C
:10330000C217D30728F4319718F00D900992F5CF22
:10331000B5CFEF91FF9185E10895A3E003DE4091E1
:103320004A01463021F04430E1F00C94D80EA3302D
:1033300071F5AAE8B4E04EE150916A015F73459FD0
:10334000A00DB11D009038014091680150916C01B1
:103350005093380155270E948239009238010C940D
:10336000D80EA230A1F4E0916801F6EFA0E8B7E032
:1033700050916A015F77A50F5AE060E844914C9341
:10338000F395A60FB21D5A95C9F70C94D80E17CF16
:10339000A2E0C8DDA23011F00C94AC0F0E94B7225D
:1033A000803009F00895403121F0483111F083E276
:1033B00008957091680190916A019A950E94D221B6
:1033C0000C94D80EA2E0AEDDA23011F00C94AC0F3C
:1033D0000E94B722803009F008954C3F11F087E138
:1033E0000895709049017091680190916A019A95D1
:1033F000909349010E949C2170924901803001F014
:103400000C94D80EAF3F31F42C9A2CBCACE5ACBD7B
:103410003DBC0895A7F92CBCAF73A064ACBD3DBC06
:10342000A5B1A4FBA5B90895BDB5B7FFFDCF08951B
:103430005C2F4D2FCF93DF9307D0DF91CF9108956D
:103440005091820140918301433038F4DDE0CCE3B8
:10345000C50FD41FA991BB2710C05050444058F04D
:10346000550F441F433038F4DDE0CCE3C50FD41FC3
:10347000A991B99102C082E10895409182015091D1
:103480008301430D521D409382015093830180308C
:1034900009F408954F914F910895A0EBB1E04FEFDB
:1034A00052E24D935A95E9F7C8EAD1E040E25A91C9
:1034B000503211F44A95D9F7442EA0EBB1E0C8E898
:1034C000D1E04C0EA03D28F4C41518F448814030DA
:1034D00009F408958AD04F3FE1F371D04F3FC9F30B
:1034E000403081F78FD0403069F73DD0403051F700
:1034F0000AD0403039F74991413618F04B3708F47B
:1035000040524D93DFCF4881403320F04A3310F4CE
:10351000405302C044270895642F7727219648819D
:10352000403380F04A3370F44053660F771F0B012D
:10353000660F771F660F771F600D711D640F721D78
:103540002196EDCF703029F04DE14D937D936D9331
:1035500008956A3020F04CE14D936D930895605DBD
:103560006D934CE108954881443211F04427089549
:1035700066277727219658815033B0F05A3310F4DC
:10358000505308C05A3508F05052513468F057343F
:1035900058F457535F70529544E0550F661F771FDC
:1035A0004A95D9F72196E7CF703029F04FE14D9336
:1035B0007D936D9308954EE14D936D9308954881E9
:1035C000423211F04427089521964D934991423299
:1035D00019F44D9341E00895403029F442E24D93AF
:1035E0004FEF4D9308954D93F1CF4881473211F03D
:1035F0004427089521964D9349914030E1F74FEFCC
:103600004D930895FF93EF93BF93AF935F93E6E7D6
:10361000FCE40E014591403089F0689457E0A59193
:10362000AE3239F0B991B13608F0B052AB1709F0AB
:10363000E8945A95A1F716F0E001EBCF5F91AF91B6
:10364000BF91EF91FF91403041F04D934F934881EE
:10365000403211F42196FBCF4F910895CBE8D1E091
:10366000A0EBB1E040E2E0E24993EA95E9F7A097E8
:10367000A03D29F04D91423010F04F3F11F42992B6
:103680000895403220F0403810F486D0F1CF4C310C
:1036900021F4ED91FF2719D0EBCF4D3121F4FD91AD
:1036A000ED9113D0E5CF4E3131F444E275D0ED9178
:1036B000689449D0DDCF4F3131F444E26DD0FD91B3
:1036C000ED9134D0D5CF50D0D3CFE8944FE243958D
:1036D000E051F742E0F7E05FF84D403311F063D07E
:1036E00068944FE24395E85EF340E0F7E851FC4F01
:1036F00016F0403311F057D068944FE24395E456EA
:10370000F040E0F7EC59FF4F16F0403311F04BD08A
:1037100068944FE24395EA50E8F7E65F16F04033CD
:1037200009F041D040E34E0F3ED00895E8944F2F6A
:1037300042954F7011F012D068944F2F4F700EF0D9
:1037400011F00CD068944E2F42954F700EF011F08E
:1037500005D068944E2F4F7001D00895405D4A33D4
:1037600008F0495F20D00895E6E7FCE45591503019
:1037700009F40895451711F03796F8CF5F9357E095
:1037800045914E3209F00FD05A95D1F75F915C31D7
:1037900010F040E208D008954993CB3A18F02992EE
:1037A0004F914F9108954993CB3A28F029924F9128
:1037B0004F914F914F910895A0914A01A0937E019E
:1037C000AA270E94A131A0913801A0937A01A0916B
:1037D0001B01A0937D01A0913601A0937901209255
:1037E0003601E8EDF1E0CCE3D7E0BEE2AEE1419195
:1037F0004993AA95E1F7BA95C9F70895A0917E017A
:103800000E94A131A0917D01A0931B01A0917A019A
:10381000A0933801A0917901A0933601ECE3F7E081
:10382000C8EDD1E0E2CFC6E1D4E0E8ECF6E041B18A
:1038300050B168E0A9E4BFEA469510F4AFE4BFE2F6
:10384000A993B193A0E3B0E8569510F4A1E3BEE4C8
:10385000AD8FB58F6A9571F70895452FA6E10E9447
:1038600010324F5B0E941B334DE30E941B33A7E1D4
:103870000E941032C0EADCE0C50FD21DC50FD21D78
:10388000A991B9919DE00E9438320895A3E10E9468
:10389000C634A5E0C62FCA95AC9FCCEFDCE0C00DC6
:1038A000D11DA881A7FF09C00E94AD34FF43414C40
:1038B0004C202000A981AF770DC00E94AD34FF4697
:1038C0004F5220004A8146954F5B0E941B330E9455
:1038D0001A33A981BB27A39592E00E9438324AE3AC
:1038E0000E941B33BB27A881AF770E94383208950E
:1038F00020921B019927A7E00E9410320E94A83253
:103900000E94AD34120042495420303132333435F4
:10391000363700000E94AD341300444952000E9423
:10392000AD3414004C455600EAE0FCE30E94153922
:10393000A5E00E9410320E94AD3400004156522D85
:1039400043686970426173696332204D4F4E202095
:1039500020205000409143014F5C0E941B330E9485
:10396000AD34FF3A000092E0BB27AC2DA3950E9436
:1039700038320E94AD34FF3A0000BB27AD2DA3952D
:103980000E943832EBE8F1E0C6EFD1E0AEE141EF62
:10399000B191B03031F0BE8F4CAF4993AA95C1F7C9
:1039A00006C0B0E2BE8F4CAF4993AA95D1F7A7E10C
:1039B0000E941032C0E0D4E0E1E1F0E10E94D7358E
:1039C0009DE050E0452F4C5FB42FAA270E94C634DB
:1039D00044DF53955D30B1F7452F4950B42FA9E02E
:1039E0000E94C6343ADF53955A31B1F7A7E30E94DB
:1039F0001032C3E1D4E0EDE1F0E10E94D7350E943E
:103A0000AD340413535441434B3A00009927BB276C
:103A1000A09180010E9438326CE0C0918001C617ED
:103A200020F0C61BB4E0B60F31DF6A95B1F70895F8
:103A30004F935F936F937F93EF93FF93CF93DF93B6
:103A4000AF93BF93AF92BF928F939F93B5DE06DE85
:103A50004FDF31D08827A09139014D3E11F4A1608C
:103A600014C0413F11F4AA2710C0423F11F4A460D2
:103A70000CC0433F39F4C2DE0E941337AA270E94CC
:103A8000A131E6CF443F29F71FC0A09339014091EF
:103A900022014030E1F7B2DE9F918F91BF90AF904D
:103AA000BF91AF91DF91CF91FF91EF917F916F9196
:103AB0005F914F91089520922301B5DE409123013B
:103AC0004030D9F30C94C0370E941A3770E0442478
:103AD00025D0ECEEFBE30E9415390E9413374D3ED2
:103AE00011F4A160D2CF443F19F40E941A37B0CF2D
:103AF000463E31F4703069F37A950E941A37E8CF68
:103B0000473E31F47A3028F773950E941A37E0CF98
:103B1000433FF9F643940E941A37DACFA7E00E9498
:103B200010320E94A8320E94AD3400004156522D3E
:103B300043686970426173696332204172726179CE
:103B4000205669657700A0E60E9410320E94AD34CD
:103B50000200416472202000A0E50E9410320E9401
:103B6000AD34020520202020202020202044617434
:103B7000612020202020202020202020000060E440
:103B8000679FCCE3DDE0C00DD11DF00163E0A0E054
:103B9000B62F0E94C634A6E00E941032DF0191E0E9
:103BA0000E949332A5E0B62F0E94C634A5E00E9481
:103BB000103290E058E0A991B0E00E949332442D79
:103BC00040FF0BC0A7E10E941032219749910E944B
:103BD0001B33A5E00E94103202C00E941A335A958E
:103BE00051F738966395633191F6089520457869C9
:103BF000742020202020202020202020202020434E
:103C000068617220204D6F6E2020204578697420F5
:103C10002020476F2020205374657020205669654E
:103C200077202041727261792092360120924A01F8
:103C3000A5E00E941032C0E0D0E0EDE1F6E10E9484
:103C40005236A0E50E9410320E94AD340102444673
:103C50004C4153482073697A653A20000E94D12272
:103C60004F3749F40E94AD34FF353132204B694261
:103C70007974650011C04F3F41F40E94AD34FF31AB
:103C8000204D69427974650007C00E94AD34FF3051
:103C900020427974650013C00E94C2224130D1F0E5
:103CA000E4ECFEE3E8940E94C238413009F434C0E9
:103CB000453009F4B9CF423099F733D0B5CFE0E0C1
:103CC000FFE3E8940E94C238413009F425C0453032
:103CD000B1F7AACFE8E8FEE3E8940E94C238413089
:103CE00009F41AC0473019F40E949E1F9DCF4A3034
:103CF00011F417D099CF423011F46DD095CF4330E5
:103D000019F40E94F71F90CF443019F40E944B2001
:103D10008BCF4530F9F688CFA0912201A030E1F792
:103D200008950E94CC3B4F466F726D6174204D65C3
:103D30006469756D3F00413009F00895A6E20E9464
:103D40001032C2E0D8E0EBE1FCE00E9423360E9492
:103D5000AD340903466F726D617474696E672E2EFF
:103D60002E202020202020000E94AD340B030000D4
:103D70000E94D422803001F50E94AD340903466FC1
:103D8000726D617474696E672E2E2E20446F6E659D
:103D90002100A2E70E9410320E94AD340B032020C4
:103DA00020507265737320616E79206B65792120D4
:103DB00020000E94133708950E94AD340903466F16
:103DC000726D617474696E672E2E2E204572726F4B
:103DD00072210000DECFA0E60E941032C4E0D8E0DD
:103DE000E9E1FDE00E9423360E94AD3409054176E9
:103DF00061696C61626C653A00000E94AD340A052D
:103E000046696C65733A20009CE00E94B422DF93FF
:103E1000CF93DF010E9438320E94AD34FF202F0083
:103E20000E94D122A42FB0E011960E9438320E9445
:103E3000AD340B05426C6F636B733A00AF91BF9169
:103E40000E9438320E94AD34FF202F000E94BC2215
:103E5000A0EFA49FD0011197B03009F413970E94EE
:103E60003832A6E00E9410320E94AD340C052020AA
:103E700020507265737320616E79206B6579212003
:103E800020000E9413370895204578697420204946
:103E90006E666F204261636B7570526573746F72EA
:103EA00052657363616E20202020202044656C657C
:103EB0007465202020202020202020202020466FF4
:103EC000726D6174204578697420466F726D6174FB
:103ED00020202020202020202020202052657363D5
:103EE000616E202020202020202020202020202043
:103EF00020202020202020202020202020202020C2
:103F00002045786974202020202020202020202097
:103F1000202020202020202052657363616E202005
:103F20002020202020202020202020202020202091
:103F300020202020202020202020202077270FD183
:103F4000A4E00E941032C1E0D2E0ECE1F5E10E9471
:103F50005236A0E40E9410320E94AD340302446540
:103F60006C6574652066696C6500B4D070936801F7
:103F7000FED24C3FD1F350D1413019F4A72FB9D222
:103F800007D308957727EBD0A4E00E941032C1E058
:103F9000D2E0ECE1F5E10E945236A0E40E9410323A
:103FA000A0E1A0936C010E94AD34030253617665D9
:103FB00020500000C0D28ED070936801D8D2403E0D
:103FC00030F4403171F0483161F0F6D0DCCFCCD222
:103FD000D03021F4CC3010F429D1D5CF8AD2ACD155
:103FE00008950ED1413079F684D2B2D10895772761
:103FF000B6D0A4E00E941032C1E0D2E0ECE1F5E1DD
:104000000E945236A0E40E941032A2E1A0936C01FB
:104010000E94AD3403024261636B757000005AD098
:1040200070936801A4D2403920F4423161F0C4D0C9
:10403000DFCF9AD2D03021F4C03610F4F7D0D8CFE9
:1040400058D21CD20895DCD0413091F652D222D2FF
:104050000895772784D0A4E00E941032C1E0D2E016
:10406000ECE1F5E10E945236A0E40E9410320E9479
:10407000AD3403024C6F6164205000005CD22AD042
:104080007093680174D2403121F0483111F0A2D010
:10409000E1CF86D10895772762D0A4E00E94103244
:1040A000C1E0D2E0ECE1F6E10E945236A0E40E94C9
:1040B00010320E94AD340302526573746F72650052
:1040C00009D07093680153D2423111F08ED0E4CF01
:1040D000F9D108957727B5D001D10E9413374D3E0D
:1040E00021F425D14F914F9108954A3E09F4089546
:1040F000403E19F405D17727EECF413E21F400D19F
:1041000070917001E8CF443E49F4703031F3F8D03B
:104110007150472F4F704F30F1F2DECF453E59F4CA
:1041200040917001471709F4D8CFEAD07395472F13
:104130004F7089F2D1CF463E29F4703170F2E0D051
:104140007051C9CF473E51F4409170014F3031F06A
:104150004051471718F0D4D0705FBDCFBECF0E943A
:10416000D122403019F44F914F911BC04093700100
:104170000E94EA360E94EA3605D2413019F04F918A
:104180004F9101C008950E94A33B4F44464C4153B8
:1041900048206E6F7420666F726D61747465640080
:1041A00008950E94A33B4F44464C415348206572FA
:1041B000726F7221000008950E94A33B4F43616E0D
:1041C000206E6F742073617665206F6E207468694D
:1041D000730008950E94A33B4F4E6F204241534904
:1041E000432066696C65000008950E94A33B4F4E12
:1041F0006F204241434B55502066696C650008951D
:104200000E94CC3BC04F76657277726974652066F8
:10421000696C653F000008950E94CC3B4F44656C7B
:104220006574652066696C653F0008950E94A33B34
:104230004F4E6F207370616365206C65667400007B
:1042400008955F936F937F93A72FA07FA0937C0126
:10425000A0917C01AF70AB5FBA2FA4E00E94C6347E
:10426000A6E00E941032A0917C01BB2795E00E943D
:1042700038320E941A33A5E00E941032A0917C01CE
:10428000A093680174D1ABD04F3F11F1A0917C0194
:104290000E94CB41C8E8D1E00E941A335CE05F93F2
:1042A0004991403808F04EE2403208F440E20E9462
:1042B0001B335F915A9599F7A0917C01A395A09328
:1042C0007C01AF7009F0C4CF7F916F915F91089529
:1042D0005DE00E941A335A95E1F7EECF4F935F935A
:1042E000C4E2D5E0472F4F705EE1459FC00DD11D60
:1042F00052EF47E159934A95E9F75F914F9108953D
:104300004F935F93C4E2D5E0472F4F705EE1459F26
:10431000C00DD11D5CE044E059934A95E9F75AE09D
:1043200043E159934A95E9F75F914F910895A09120
:104330002201A030E1F70895709368014CE04093AA
:104340006A0140E140936C0120D1803009F029CF0F
:104350007093680190914901ECE0F0E997709295B3
:1043600040EC949FE00DF11D04913C9740E10E3428
:1043700009F448E10E94F73E40E04F9300E0CCE3AF
:10438000DFE0159119930A95E1F740936A0142E045
:1043900040936C0103D14F9143954C3071F70895D0
:1043A000909149019770E0E0F0E9929540EC949F7C
:1043B000E00DF11D40E04F9340936A0142E04093CD
:1043C0006C0170936801E7D0CCE3DFE00E9476795E
:1043D00032964F9143954C3071F77894089540315F
:1043E00039F40E94AD34FF4241533A0040E1089550
:1043F000423139F40E94AD34FF4255503A0042E157
:104400000895443139F40E94AD34FF5553523A00B7
:1044100044E10895463139F40E94AD34FF434838F1
:104420003A0046E10895483139F40E94AD34FF4224
:10443000494E3A0048E108954A3139F40E94AD34BA
:10444000FF47504F3A004AE108954C3139F40E9439
:10445000AD34FF53414D3A004CE108954E3139F4EB
:104460000E94AD34FF4C424C3A004EE108950E9448
:10447000AD34FF2D2D2D2D004FEF08957093680161
:1044800040E640936A0142E140936C017ED0803067
:1044900009F087CE709368014427E0E0F0E94F937C
:1044A000CCE3DFE00024159019920A94E1F74093E1
:1044B0006A0142E040936C0171D04F9143954036C0
:1044C00071F7089540E0E0E0F0E94F9340936A010E
:1044D00042E040936C01709368015DD0CCE3DFE073
:1044E0000E94767932964F914395403671F77894D1
:1044F00008950E9424014F93409138014093710127
:104500004CE440933801C6E0DAE0E7E1FCE00E94C9
:1045100023360E94AD340B0757726974696E6720A9
:10452000646174612E2E2E00409171014093380118
:104530004F910C941D01CAE3CAE340914901942FA5
:104540004F5C499340E249934BE5499340913501D3
:104550004F934068409335010E94A8794DE54993F7
:104560004F914093350108950E945D4008950E9447
:1045700025410E94FB3E08950E94A43E08950E949A
:10458000293F08950E943C4008950E94BA40089532
:104590000E942D4108950E94A34108950E9449411F
:1045A00008950E94B23E08950E94D63F0895A1E06A
:1045B0000E947A382092360120924A01A7E00E9498
:1045C0001032C0E0D0E0EDE1F6E10E945236A0E703
:1045D0000E9410320E94AD3401024156522D4368B0
:1045E000697042617369633220636F6E66696770D8
:1045F00061676500A7E00E9410320E94AD3414018B
:10460000436865636B73756D3A2000006AD168D0AA
:10461000E4E4F9E4E8940E94C238413011F40C94C7
:104620000000423059F44091180150E24527409370
:1046300018010E940B790E946C24E9CF433071F479
:1046400040911801542F53955170487F452B40934A
:1046500018010E940B790E946C24D9CF443059F480
:104660004091180150E14527409318010E940B79B1
:104670000E946C24CCCF453059F44091180158E089
:104680004527409318010E940B790E946C24BFCFEC
:10469000473049F440916501542F43954770587F46
:1046A00040936501F0CF483051F440911801405CCF
:1046B000409318010E940B790E946C24A8CF4930C6
:1046C00051F4409165014058409365010E940B7977
:1046D0000E946C249CCF4A3011F40E94432E67CF75
:1046E000A6E00E9410320E94AD3403014B6579624E
:1046F0006F617264206C61796F75743A00000E947A
:10470000AD34050153657269616C20737065656431
:104710003A000E94AD340701493243207370656549
:10472000643A00000E94AD3409015350492073706F
:104730006565643A00000E94AD340B014545505256
:104740004F4D20616464726573733A000E94AD340A
:104750000D014C696E6520456E643A000E94AD34CF
:104760000F0153657269616C20696E7465726661D0
:1047700063653A00A1E70E9410327091180175FD3F
:104780000AC00E94AD3403124445202851574552B7
:10479000545A290009C00E94AD34031255532028F1
:1047A000515745525459290070FD0AC00E94AD343A
:1047B000051220313230302042707320200009C0B1
:1047C0000E94AD3405122032343030204270732004
:1047D000200074FD0AC00E94AD3407122020313041
:1047E00030206B487A20200009C00E94AD340712A7
:1047F0002020343030206B487A20200073FD0AC01E
:104800000E94AD3409122020202035204D487A2006
:10481000200009C00E94AD34091220203135362015
:104820006B487A202000707C51F40E94AD340D1248
:104830002020206E6F6E65202020200021C0703463
:1048400051F40E94AD340D12206F6E6C79204C46ED
:104850002020200015C0703851F40E94AD340D1294
:10486000206F6E6C792043522020200009C00E94E6
:10487000AD340D12202043522B4C46202020200026
:104880007091650177FD0AC00E94AD340F1220209F
:1048900073696D706C652020200009C00E94AD34E2
:1048A0000F12207374616E646172642020000E9494
:1048B000AD340B12202020202000472F4770405D90
:1048C0000E941B330E94AD34FF20202020200000D6
:1048D000A7E00E9410320895A0912201A030E1F7D4
:1048E0000895AA27BB27CC27DD27EE27FF271590A1
:1048F00042E0149EA00DB11DC21DD21D459147E09E
:10490000149EA00DB11DC21DD21DFE3881F7EE27E9
:10491000F0EF459141E7149EB01DC11DD21D459198
:1049200047E0149EB01DC11DD21DF03091F7BF931A
:10493000AF93DE019FE00E949332AF91BF910E943E
:1049400093320895204578697420204B6579622060
:1049500020536572202020493243202020535049A3
:104960002020202020202020454550524F4D204C13
:10497000696E6520536572696E7420436C6F6E6555
:10498000AEE0A0933801C1E0D4E0ECE1F2E10E9496
:1049900023360E94AD34050500000E947C020E946F
:1049A000AD34060320202020202863292032303017
:1049B000362D3230303920202020202000000E9467
:1049C000AD340703202020206279204A6F6572678A
:1049D00020576F6C6672616D202020200000A2EAD3
:1049E000A09338010E94AD3409032020202020200C
:1049F00044656469636174656420746F20202020BD
:104A0000202000000E94AD340A03466C6F72696179
:104A10006E2C204572696B20616E64204469616E62
:104A2000612E0000AEE0A09338010E94AD340C026C
:104A30005468697320736F66747761726520697357
:104A4000206C6963656E736564000E94AD340D046B
:104A5000756E64657220746865207465726D73206C
:104A60006F662074686520000E94AD340E04474EC6
:104A700055205055424C4943204C4943454E5345DF
:104A800020562E3320000E94AD340F03557365204D
:104A9000697420617420796F7572206F776E20724F
:104AA00069736B210000A2ECA09338010E94AD3421
:104AB000110720505245535320414E59204B455920
:104AC00020000E941337089561E00E94AB38509196
:104AD00022015D3E09F408954531B1F790914901F5
:104AE000E0E0F0E99770929540EC949FE00DF11DA5
:104AF000CCE3DDE050E0459149935A95E1F7CCE3F2
:104B0000DDE00E94CB3D0E94AB38509122015D3E1A
:104B100011F34630A1F76395CCEBDDE00E94CB3D6D
:104B20000E94AB38509122015D3EA9F24630A1F7B8
:104B300063956931E9F644E00E948F3808959091B9
:104B400049019770E0E0F0E9929540EC949FE00D08
:104B5000F11D45E10E948F3860E06F93CCE3DFE008
:104B60000E94A83D803041F0813051F1883241F1FE
:104B700045E10E948F38F2CF46E00E948F38CCEB9F
:104B8000DFE00E94A83D803041F08130C9F08832DA
:104B9000B9F045E10E948F38F2CF0E94767978947F
:104BA000329646E00E948F386F9163956C30A9F67B
:104BB0000E949B384430E1F746E00E948F38089508
:104BC0006F91089561E00E94AB38509122015D3EE3
:104BD00009F408954531B1F7A0E8762F7A95A79F9B
:104BE000E001ACE3BDE070E80E945E3E4D937A9533
:104BF000D9F7CCE3DDE00E94CB3D0E94AB38509169
:104C000022015D3E31F34630A1F763956F3021F705
:104C100044E00E948F38089545E10E948F3860E09B
:104C20006F93CCE3DDE00E94A83D803031F0883204
:104C300001F145E10E948F38F4CFA0E8762F7A95F4
:104C4000A79FE001ACE3BDE070E84D910E94673E94
:104C50007A95D9F746E00E948F386F9163956E3050
:104C6000F9F60E949B384430E1F746E00E948F3805
:104C700008956F91089502414253282E2E2E03531A
:104C8000474E282E2E2E04535152282E2E2E054EDE
:104C90004F54282E2E2E06524E44282E2E2E0741DB
:104CA0004443282E2E2E08494E282E2E2E2E0958EB
:104CB0005045454B282E0A54454D50282E2E0B4C5E
:104CC0004F282E2E2E2E0C4849282E2E2E2E0D4BE0
:104CD0004559282E2E2E0E455045454B282E0F4562
:104CE0005252282E2E2E104152282E2E2E2E115387
:104CF000494E282E2E2E12434F53282E2E2E134669
:104D000054595045282E144653495A45282E1550BB
:104D100053544154282E16535049282E2E2E174DE9
:104D2000454E55282E2E185642595445282E1958AE
:104D3000524543282E2E1A4646494E44282E80506E
:104D400052494E542E2E81434C532E2E2E2E8247E6
:104D50004F544F2E2E2E83424F582E2E2E2E8441EE
:104D6000434F50592E2E8553594E432E2E2E864595
:104D70004E442E2E2E2E8742434F50592E2E8854AD
:104D800048454E2E2E2E89504F532E2E2E2E8A4EB3
:104D90004F54452E2E2E8B4F4E53594E432E8C5230
:104DA000524541442E2E8D5257524954452E8E471E
:104DB0004F5355422E2E8F52455455524E2E9056DB
:104DC0004D4F44452E2E914E4558542E2E2E92492D
:104DD0004E5055542E2E93504C4F542E2E2E9457E9
:104DE0004149542E2E2E95545345542E2E2E965412
:104DF0004745542E2E2E974653454C454354984FC5
:104E00004E4552522E2E99535055542E2E2E9A53B3
:104E10004745542E2E2E9B45504F4B452E2E9C47DA
:104E200045545049582E9D434952434C452E9E436C
:104E30004F4C4F522E2E9F424F524445522EA04669
:104E40004F4E542E2E2EA150554D502E2E2EA25880
:104E5000504F4B452E2EA356504F4B452E2EA44C53
:104E6000494D49542E2EA547455443484152A64426
:104E7000524157544F2EA7504C41592E2E2EA85315
:104E800050524954452EA95343524F4C4C2EAA42DE
:104E90005245414B2E2EAB464153542E2E2EAC5331
:104EA0004C4F572E2E2EAD445241572E2E2EAE492A
:104EB000434F4D4D2E2EAF444154412E2E2EB04324
:104EC000544558542E2EB146524541442E2EB246DA
:104ED00057524954452EB343424F582E2E2EB447B5
:104EE000455441545452B54644454C455445B64644
:104EF000424F582E2E2EB750414C45545445B8467B
:104F00004F522E2E2E2EB949462E2E2E2E2EBA441C
:104F100049522E2E2E2EBB4F55542E2E2E2EBC46D1
:104F2000434952434C45BD414C4552542E2EBE463A
:104F3000435245415445BF41534B2E2E2E2EC03F68
:104F40002E2E2E2E2E2EC15853454E442E2EC247A5
:104F50004F2E2E2E2E2EC3544F2E2E2E2E2EC44CC0
:104F60004F4144502E2EC643434841522E2EC74235
:104F7000432E2E2E2E2EC853415645502E2ECA4E4D
:104F80004F2E2E2E2E2ECC5252442E2E2E2ECD5261
:104F900057522E2E2E2ECE474F532E2E2E2ECF5220
:104FA00045542E2E2E2ED0564D2E2E2E2E2ED2493C
:104FB0004E502E2E2E2ED3504C2E2E2E2E2ED74629
:104FC00053454C2E2E2EDC4750582E2E2E2EDD43D0
:104FD000492E2E2E2E2EDE434F4C2E2E2E2EDF420D
:104FE0004F2E2E2E2E2EE258502E2E2E2E2EE356E3
:104FF000502E2E2E2E2EE44C494D2E2E2E2EE547D1
:1050000043482E2E2E2EE644544F2E2E2E2EE8539D
:1050100050522E2E2E2EED44522E2E2E2E2EEE4996
:10502000432E2E2E2E2EEF44412E2E2E2E2EF146C6
:1050300052442E2E2E2EF24657522E2E2E2EF4474E
:1050400041542E2E2E2EF54644454C2E2E2EF75032
:10505000414C2E2E2E2EFC4643492E2E2E2EFE4641
:1050600043522E2E2E2E002E2E2E2E2E2E2EA09180
:105070001401B0911501ED01E2EBF2E0CE0FDF1F5C
:10508000F6EFE0911A01FE0F7F934F92EEE14E2E64
:105090006991ED915491762F7295762757FD672788
:1050A00068B9ED91000056FD76B9049055FD76B9CA
:1050B0006991162E54FD76B91294162653FD76B9D1
:1050C00007FC61254A9452FD76B9502D712D41F7A8
:1050D00060911B0168B94F907F91EE91F0911A0198
:1050E000F395FA3029F4FF27A0931401B09315012A
:1050F000F0931A010C949E30A0911401B091150107
:10510000D0910001C0910101C295DC0FDE7EE5E186
:1051100010901B01FD914D2FF0FD429548B9000004
:105120004D2FF1FD429548B900004D2FF2FD4295FB
:1051300048B900004D2FF3FD4295000048B96D2F8E
:105140004D2FF4FD429548B9CD91F5FD62955D2F47
:1051500068B9F6FD52956D2F4D2F58B9F7FD629540
:10516000C0FD4295000068B9FC2FEA95B9F618B861
:10517000EE91F0911A01F395F23029F4FF27A093F4
:105180001401B0931501F0931A010C949E30A09174
:105190001401B0911501D1E0FEE110901B01ED91D9
:1051A000CE2FC370588158B9CE2FC695C695C370FF
:1051B0005881E29558B9CE2FC3705881CE2FC6952D
:1051C00058B9C695C3705881ED91CE2F58B9C370A8
:1051D0005881FA9541F718B8EE91F0911A01F395BC
:1051E000F33029F4FF27A0931401B0931501F09335
:1051F0001A010C949E30A0911401B09115010F93E7
:1052000010901B01EAE2D1E0CD91C6950C2FC2951A
:10521000CF70F881F8B9C02F0000CF70F88100007E
:1052200000000000F8B9CD91C6950C2FC295CF7043
:10523000F881EA9579F718B811970F91F0911A0152
:10524000F395F43029F4FF27A0931401B0931501CE
:10525000F0931A010C949E30A0911401B0911501A5
:10526000D0910001C0910101C295DC0FDE7EE0E12A
:1052700010901B01FD914D2FF0FD429548B90000A3
:10528000000000004D2FF1FD429548B900000000DC
:1052900000004D2FF2FD429548B9000000004D2F4F
:1052A000F3FD4295000048B9000000006D2F4D2F1E
:1052B000F4FD429548B90000CD91F5FD62955D2F52
:1052C00068B900000000F6FD52956D2F4D2F58B9BA
:1052D000F7FD6295C0FD42950000000068B9FC2F03
:1052E00000000000EA9551F6000018B8EE91F09128
:1052F0001A01F395F33029F4FF27A0931401B0931A
:105300001501F0931A010C949E30A0911401B091F4
:105310001501C0914D01D82DF6EFE0911A01FE0F55
:10532000E395E0931A01EA3088F1EC3069F5939641
:10533000A0931401B093150120921A01DC3031F4CE
:10534000D0914C01D0934D010C949E30D83189F40A
:10535000A1E4B2E0C0913A01D3E2CD9FA00DB11D0E
:10536000CFE0A0931401B0931501C0934D010C94AC
:105370009E30D83D49F4CBE4AEE1B2E0A0931401F5
:10538000B0931501C0934D010C949E300F931F9361
:105390002F93D83D28F4DC2F0C2F1C2F2C2F05C069
:1053A00029E61DE208E8DCECCBE46C2F7C2F72953B
:1053B000ED91E7FD6727EF775491ED9168B9172ECE
:1053C00056FD16B86C2F7C2F729555FD16B8E7FD6B
:1053D000672754FD16B8EF77000053FD16B8049008
:1053E00052FD16B8502DED9168B9172E56FD16B81E
:1053F0006C2F7C2F729555FD16B8E7FD672754FD7D
:1054000016B8EF77000053FD16B8049052FD16B899
:10541000502DED9168B9172E56FD16B86C2F7C2FC4
:10542000729555FD16B8E7FD672754FD16B8EF775E
:10543000000053FD16B8049052FD16B8502DED91A2
:1054400068B9172E56FD16B86C2F7C2F729555FD36
:1054500016B8E7FD672754FD16B8EF77000053FD37
:1054600016B8049052FD16B8502DED9168B9172E5C
:1054700056FD16B86C2F7C2F729555FD16B8E7FDBA
:10548000672754FD16B8EF77000053FD16B8049057
:1054900052FD16B8502DED9168B9172E56FD16B86D
:1054A0006C2F7C2F729555FD16B8E7FD672754FDCC
:1054B00016B8EF77000053FD16B8049052FD16B8E9
:1054C000502DED9168B9172E56FD16B86D2F7D2F12
:1054D000729555FD16B8E7FD672754FD16B8EF77AE
:1054E000000053FD16B8049052FD16B8502DED91F2
:1054F00068B9172E56FD16B86D2F7D2F729555FD84
:1055000016B8E7FD672754FD16B8EF77000053FD86
:1055100016B8049052FD16B8502DED9168B9172EAB
:1055200056FD16B86D2F7D2F729555FD16B8E7FD07
:10553000672754FD16B8EF77000053FD16B80490A6
:1055400052FD16B8502DED9168B9172E56FD16B8BC
:105550006D2F7D2F729555FD16B8E7FD672754FD19
:1055600016B8EF77000053FD16B8049052FD16B838
:10557000502DED9168B9172E56FD16B86D2F7D2F61
:10558000729555FD16B8E7FD672754FD16B8EF77FD
:10559000000053FD16B8049052FD16B8502DED9141
:1055A00068B9172E56FD16B86D2F7D2F729555FDD3
:1055B00016B8E7FD672754FD16B8EF77000053FDD6
:1055C00016B8049052FD16B8502DED9168B9172EFB
:1055D00056FD16B86D2F7D2F729555FD16B8E7FD57
:1055E000672754FD16B8EF77000053FD16B80490F6
:1055F00052FD16B8502DED9168B9172E56FD16B80C
:10560000602F702F729555FD16B8E7FD672754FD82
:1056100016B8EF77000053FD16B8049052FD16B887
:10562000502DED9168B9172E56FD16B8602F702FCA
:10563000729555FD16B8E7FD672754FD16B8EF774C
:10564000000053FD16B8049052FD16B8502DED9190
:1056500068B9172E56FD16B8602F702F729555FD3C
:1056600016B8E7FD672754FD16B8EF77000053FD25
:1056700016B8049052FD16B8502DED9168B9172E4A
:1056800056FD16B8602F702F729555FD16B8E7FDC0
:10569000672754FD16B8EF77000053FD16B8049045
:1056A00052FD16B8502DED9168B9172E56FD16B85B
:1056B000602F702F729555FD16B8E7FD672754FDD2
:1056C00016B8EF77000053FD16B8049052FD16B8D7
:1056D000502DED9168B9172E56FD16B8602F702F1A
:1056E000729555FD16B8E7FD672754FD16B8EF779C
:1056F000000053FD16B8049052FD16B8502DED91E0
:1057000068B9172E56FD16B8612F712F729555FD89
:1057100016B8E7FD672754FD16B8EF77000053FD74
:1057200016B8049052FD16B8502DED9168B9172E99
:1057300056FD16B8612F712F729555FD16B8E7FD0D
:10574000672754FD16B8EF77000053FD16B8049094
:1057500052FD16B8502DED9168B9172E56FD16B8AA
:10576000612F712F729555FD16B8E7FD672754FD1F
:1057700016B8EF77000053FD16B8049052FD16B826
:10578000502DED9168B9172E56FD16B8612F712F67
:10579000729555FD16B8E7FD672754FD16B8EF77EB
:1057A000000053FD16B8049052FD16B8502DED912F
:1057B00068B9172E56FD16B8612F712F729555FDD9
:1057C00016B8E7FD672754FD16B8EF77000053FDC4
:1057D00016B8049052FD16B8502DED9168B9172EE9
:1057E00056FD16B8612F712F729555FD16B8E7FD5D
:1057F000672754FD16B8EF77000053FD16B80490E4
:1058000052FD16B8502DED9168B9172E56FD16B8F9
:10581000612F712F729555FD16B8E7FD672754FD6E
:1058200016B8EF77000053FD16B8049052FD16B875
:10583000502DED9168B9172E56FD16B8612F712FB6
:10584000729555FD16B8E7FD672754FD16B8EF773A
:10585000000053FD16B8049052FD16B8502DED917E
:1058600068B9172E56FD16B8622F722F729555FD26
:1058700016B8E7FD672754FD16B8EF77000053FD13
:1058800016B8049052FD16B8502DED9168B9172E38
:1058900056FD16B8622F722F729555FD16B8E7FDAA
:1058A000672754FD16B8EF77000053FD16B8049033
:1058B00052FD16B8502DED9168B9172E56FD16B849
:1058C000622F722F729555FD16B8E7FD672754FDBC
:1058D00016B8EF77000053FD16B8049052FD16B8C5
:1058E000502DED9168B9172E56FD16B8622F722F04
:1058F000729555FD16B8E7FD672754FD16B8EF778A
:10590000000053FD16B8049052FD16B8502DED91CD
:1059100068B9172E56FD16B8622F722F729555FD75
:1059200016B8E7FD672754FD16B8EF77000053FD62
:1059300016B8049052FD16B8502DED9168B9172E87
:1059400056FD16B8622F722F729555FD16B8E7FDF9
:10595000672754FD16B8EF77000053FD16B8049082
:1059600052FD16B8502DED9168B9172E56FD16B898
:10597000622F722F729555FD16B8E7FD672754FD0B
:1059800016B8EF77000053FD16B8049052FD16B814
:10599000502DED9168B9172E56FD16B8622F722F53
:1059A000729555FD16B8E7FD672754FD16B8EF77D9
:1059B000000053FD16B8049052FD16B8502DED911D
:1059C00028B82F911F910F910C949E30A091140133
:1059D000B0911501EAE8F4E0C0911A01D3E0CD9F3F
:1059E000E00DF11D7F936EE17EE1CBE1D1E05881C6
:1059F000507F452F4295542B588358B952954D915D
:105A00004F7358B95991469F58B95295EF0100000C
:105A100058B9C00DD11D599158B952957A950000C9
:105A2000000058B9599149F7000058B95295609152
:105A30001B01000058B959917F9158B95295F091C6
:105A40001A01F39558B90000000068B9FA3029F43A
:105A5000FF27A0931401B0931501F0931A010C9441
:105A60009E30A0911401B0911501ED01E2EBF2E03E
:105A7000CE0FDF1FF7E0E0911A01E395E0FBE6951A
:105A8000FE0F7F934F92EEE14E2E6991ED91E7F973
:105A90005081762F7295762757FD672768B9ED916B
:105AA000E7F956FD76B90080000055FD76B9699199
:105AB000162E54FD76B91294162653FD76B907FCBE
:105AC00061254A9452FD76B9502D712D39F76091B8
:105AD0001B0168B94F907F91EE91F0911A01F395F7
:105AE000FA3029F4FF27A0931401B0931501F09325
:105AF0001A010C949E30A8EDB1E0C4E1D2E080928E
:105B00001A010C944028A6EFB1E0C2E3D2E0425D56
:105B100040931A010C944028482D4A5008F4EBCFCA
:105B2000423D08F0F0CF58E14695A0E5B2E0A40F61
:105B3000B21D4C91459FA9EBB2E0A00DB11DCFE97C
:105B40004D915D91C395C41731F000000000000035
:105B5000C215C1F792C04D9158B96D91C395C41744
:105B600031F00000529558B9C215C1F786C04D9169
:105B700068B95D91C395C41731F00000629568B9AA
:105B8000C215C1F77AC04D9158B96D91C395C4172C
:105B900031F00000529558B9C215C1F76EC04D9151
:105BA00068B95D91C395C41731F00000629568B97A
:105BB000C215C1F762C04D9158B96D91C395C41714
:105BC00031F00000529558B9C215C1F756C04D9139
:105BD00068B95D91C395C41731F00000629568B94A
:105BE000C215C1F74AC04D9158B96D91C395C417FC
:105BF00031F00000529558B9C215C1F73EC04D9121
:105C000068B95D91C395C41731F00000629568B919
:105C1000C215C1F732C04D9158B96D91C395C417E3
:105C200031F00000529558B9C215C1F726C04D9108
:105C300068B95D91C395C41731F00000629568B9E9
:105C4000C215C1F71AC04D9158B96D91C395C417CB
:105C500031F00000529558B9C215C1F70EC00000CE
:105C6000000068B900000000C395C41700000000E0
:105C7000629568B9C215C1F700C050911B010000C0
:105C8000000058B95BC20E94CC3B6F436C6F6E65DD
:105C90002073797374656D3F2000413009F00895D9
:105CA00065D087D0803079F078D00E94A33B4F4EEA
:105CB0006F20636F6E74726F6C6C657220666F75A7
:105CC0006E64200008958DD0803069F066D00E9407
:105CD000A33B4F4E6F204D65676136343420666FAD
:105CE000756E64000895CDD09DD0EE27FF2750E05B
:105CF00060E00590B8D00590BDD063956038C9F7D5
:105D00009ED05395A9F74CEA4ED040EA4CD04AD0E9
:105D100046EE49D00E94EA360E94EA360E94EA36F0
:105D20004CEA41D048EA3FD03DD041ED3CD00E9402
:105D3000EA360E94EA360E94EA364CEA34D044EA57
:105D400032D030D04CEF2FD00E94EA360E94EA3693
:105D50000E94EA3622D00E94A33B80537973746577
:105D60006D20636C6F6E65640000089543E54CBD63
:105D70002DBC249A2C984FEF4A95F1F72C9A4FEFAF
:105D80004A95F1F72C984FEF4A95F1F72C984FEF81
:105D90004A95F1F70E94EA3608952C9A4CE54CBDDD
:105DA0003DBC089544274EBD4DB547FFFDCF4EB5D0
:105DB000089588274CEAF7DF43E5F5DFF3DF433545
:105DC00009F081E0EFDF0895BF93AF934F93A42FC5
:105DD000BB270E9493320E941A334F91AF91BF911B
:105DE0000895882740E3DFDFDDDF40E0DCDFDADF36
:105DF0004E3111F082E0089540E3D5DFD3DF41E07A
:105E0000D2DFD0DF463911F082E0089540E3CBDFE6
:105E1000C9DF42E0C8DFC6DF493019F04A3009F077
:105E200082E008954CEABFDF40E8BDDFBBDFBADFA8
:105E30000E94EA360E94EA360E94EA3608954CE44F
:105E4000B2DF452F4695AFDF452F440F440F440F77
:105E5000440F440F440F440FA6DFA4DF0E94EA362C
:105E60000E94EA36089540E49EDF9CDF462F9BDFC8
:105E7000402D99CF48E497DF95DF462F94DF402DE2
:105E800092CF0E9424014F934091380140937101B9
:105E90004CE440933801C5E0DAE0E8E1FCE00E9420
:105EA00023360E94AD340B06436C6F6E696E67201B
:105EB00053797374656D2E2E2E00409171014093BD
:105EC00038014F910C941D0128B818954F935F939A
:105ED0006F93FF93EF93DF93CF93BF93AF930F92A3
:105EE0001F92FFB7FF9330921D01B0913D01B7FFA4
:105EF0005C98B7FD5C9A4B99BE7F4B9BB160A091BB
:105F00006501C1E0A7FDBC27B0933D01C4E1D1E02C
:105F10005F89A889E9890A881B88A00DE11DA88BE3
:105F2000E98BFFA14491AD89AF73AF3309F4452FDD
:105F30005AA54503B0E8B10DB093B300EE89FF89CF
:105F4000488D598DAA27E2FDA095E5FDA095F4FDA9
:105F5000A09557FDA095AA1FEE1FFF1F441F551FB8
:105F6000EE8BFF8B488F598F830C921CEBA9FF811E
:105F7000EF23E8B97894E9A190FC04C0F8A58F1646
:105F800008F4A9C071F4409110014F3F51F04091C5
:105F900012014A9521F4409111013092130140936E
:105FA0001201FCE0E2FFFDEE8F1639F45E98E3FF8C
:105FB000C5C0B2E8B0938000C1C0F1E1E2FFF3EFE9
:105FC0008F1639F45E9AE3FFB9C0B2ECB09380004B
:105FD000B5C0FBE1E2FFFFEF8F1621F4EFEFE09396
:105FE0004701ACC0F2E0E2FFF9EE8F1619F42092FF
:105FF0004701A4C0F9E3E2FFF7E08F1609F09EC065
:10600000A8EDA883A1E0A9832E8288249924AAE080
:10601000A9AFA5E0E2FFA39542E3E2FF4CE3BA8D0E
:10602000B395BA1731F4BB27EB8DFC8D3196EB8F0E
:10603000FC8FBA8FE885E395E41709F4EE27E8872B
:10604000FDE8E0E0A0912901A7FDB096AC89EA0F38
:10605000F21DB491B21511F0A395AC8BBAA7A09123
:106060005C01A03009F46AC0B0915D01B395B093B2
:106070005D01BA17C0F320925D01B0916401BA9539
:10608000B093640181F7E0915E01F0915F01C091EE
:106090006201D09163012196A191B191B093640105
:1060A000E0935E01F0935F019ED6FD1798F0EC1728
:1060B00088F0A0913F01A13029F4A2E020925C0178
:1060C000A0933F01E0916001F0916101E0935E01D6
:1060D000F0935F0133C0A0918400A63EE0F3A73E99
:1060E00000F0A83E00F0A93E00F0AA3E00F0E5FD59
:1060F00025C0E0913501E7FD0C948529E0914A0126
:10610000E53011F40C942C29E03011F40C9437286C
:10611000E13011F40C947C28E23011F40C94C7287F
:10612000E43011F40C94312DE63011F40C94E62C8B
:10613000E73011F40C948C2D0C94FB28A0912001D5
:10614000A5FD27C0E091C000E7FF6BC0E091C6004D
:10615000E0938101F5EFB491B0FF36C0A7FF03C013
:10616000209222015BC0E33809F4E0E1F6E84091B7
:10617000180145FDFE5FEF77A4FFA6FDF395A4FF90
:10618000A0FDE068A1FDE068E491E0932101A06238
:1061900046C0E0912101E0932201E0932301EE3E0D
:1061A00019F4A2FD0C94EF0040913901E33611F48B
:1061B000A2FD4160E03711F4A3FD4260EC3F09F419
:1061C0004460409339012AC0E03F11F4A06827C021
:1061D000E03E11F4A06423C0E23131F4A6FD1EC0FC
:1061E000A160A7FDAE7F1AC0E93521F4A260A7FD2A
:1061F000AD7F14C0E43151F4A6FD04C0A460A7FD36
:10620000AB7F0CC0A860A7FDA77F08C0E13121F4D7
:10621000A061A7FDAF7E02C020922201AF71A093C2
:1062200020014091180140FD0E94A57840FF0E9486
:10623000DA78FF91FFBF1F900F90AF91BF91CF9180
:10624000DF91EF91FF916F915F914F911895AAEBBC
:10625000A4B9AFEFA5B9A0EEA7B9A0E0A8B9A0EF87
:10626000AAB9AFEFABB9A6B1AF77A0933501B2EC45
:10627000B0938000B9E1B0938100F4E0A2FFF4E0B4
:10628000F0938700FEEFA2FFF6EFF09386002092D6
:106290008900FAE5F0938800F4E0F0938B00F8EDC4
:1062A000F0938A00A6E0A0936F00A2E0A4BDA1E055
:1062B000A5BDA1E3A7BDA3E8A093B000A1E0A09372
:1062C000B100A0E8A093B3002092B6002092C000D5
:1062D000A0E1A093C100A6E6A093C200ACE5B091F6
:1062E0001801B3FDAFE5ACBDA0E0ADBDA5E198D010
:1062F000C4E1D1E0A8EDA993A1E0A993AEE1299270
:10630000AA95E9F7AAEAA0932A01A0932C0120926A
:10631000360120921901AEE3A09328010F9300915A
:1063200035010F770093350106EE07C00F930091FA
:10633000350100680093350104EE00933C010F9194
:106340000895A0934A01A03021F0A43051F40E9496
:106350009A39ACE3A0935001AEE2A0935101A6EEAE
:1063600044C0A13069F4A8EAA0935001A4E7A09327
:106370005101A0E0A0930001A0EEA093010124C070
:10638000A23091F4A8E7A0935001ACE4A09351018E
:10639000C0E0D1E0A0E0A993A0E4A993A0EAA9936A
:1063A000A0EEA993A3EE21C0A33081F4A4E5A093AD
:1063B0005001AAE3A0935101C0E0D1E0AA27B0E1C7
:1063C000A993A05EBA95E1F7A7EE0FC0A53081F4BE
:1063D000A0E8A0935001A0E4A0935101A0E2A093F3
:1063E0000001A0EEA0930101A0ECA0933C01089550
:1063F000A63051F4ACE3A0935001AEE2A09351015A
:106400000E945C39A6EEF1CFACE3A0935001A2E06C
:10641000A09351010E94B2390E94C339A6EEE5CF84
:10642000AA0FAE7EA09338010895A295AA0FA07E70
:10643000A0931B01089548834091350147FD17C083
:1064400040914A01463099F0CF93DF935F935CE32C
:10645000C50FD21D473021F046E7C40F42E0D41FDC
:10646000409138014E7E48835F91DF91CF9108952E
:106470004F935F936F93AF93BF9340E2592F537045
:10648000523061F0533009F44BE2B7FF05C0A095DC
:10649000B095A30DB21D4DE20E941B33592F5C70C5
:1064A000692F6073E8944FE24395A051B742E0F73B
:1064B000A05FB84D5C3009F42BD04FE24395A85E45
:1064C000B340E0F7A851BC4F53FD22D0603309F42C
:1064D000AFD04FE24395A456B209E0F7AC59BF4F95
:1064E000503009F015D0603209F4A2D04FE2439544
:1064F000AA50E8F70DD0A65F603109F499D040E3C7
:106500004A0F99D0BF91AF916F915F914F910895CC
:10651000403311F068948FC091FD8DC0F6F390FF69
:10652000089588C008954F9390FF05C04B2F429562
:1065300009D04B2F07D04A2F429504D04A2F02D0C2
:106540004F9108954F70405D4A3308F0495F73C022
:1065500040914A014030D9F04430C9F0AF93BF9325
:10656000CF93DF93D1E0C8EDA7E1463009F0ACE569
:10657000BEE12992BA95E9F7AA95D1F7DF91CF91BB
:10658000AA24BB2420923701BF91AF910895AF9305
:10659000BF93CF93DF9340E2D1E0C8EDA7E1BEE126
:1065A0004993BA95E9F7AA95D1F7409138014E7E03
:1065B000A7E1BEE14993BA95E9F7AA95D1F7DF9132
:1065C000CF91AA24BB2420923701BF91AF910895A7
:1065D000AF93BF9320923701A0913601A03051F4C0
:1065E000A7E1AA24B394AB1571F7B6E1BB2ECF9304
:1065F000DF936CC0A13021F4BF91AF910C9482382D
:10660000A23059F44DE0B0911801B6FD94D44AE09F
:10661000B7FD91D4BF91AF910895A33019F4BF9104
:10662000AF910895BF91AF915AE00E94EE3D089559
:106630004CE201C040E2AF93BF93A0913701A39514
:10664000A0933701A0913601A43030F0BF91AF91F3
:10665000542F0E94EE3D0895A030A9F0A33059F4C4
:10666000A42FBB275F936F930E946E186F915F9169
:10667000BF91AF910895BF91AF91A0913601A1FF55
:106680000C948F3858C4EF93E0914A01E03029F020
:10669000E43019F0E63008F49AC0EF91CF93DF931D
:1066A0002ED496FD35C0C7DEA395AE3131F4AA27AE
:1066B000B395B73111F4B6E107C0AA2EBB2EDF9116
:1066C000CF91BF91AF910895AA2EBB2ED1E0C8ED16
:1066D0004F93A6E1BEE14E8D4993BA95E1F7AA9595
:1066E000C9F7AEE140E24993AA95E9F7D4E0CAE8D8
:1066F000A6E1BEE14E8D4993BA95E1F7AA95C9F797
:10670000AEE1409138014993AA95E9F74F91D7CF6F
:10671000AB31A8F6B23198F6AD5FAA2EEF93FF9396
:106720004F925F926F927F9270F85F93E42FF6EF33
:10673000B5E04424552466245527A491A7FD53951C
:1067400050FB40F8A6FD539550FB41F8A5FD53952D
:1067500050FB50F8A4FD539550FB51F8A3FD539501
:1067600050FB60F8A2FD539550FB61F8F395552757
:10677000A491A7FD539550FB42F8A6FD539550FBFD
:1067800043F8A5FD539550FB52F8A4FD539550FBDB
:1067900053F8A3FD539550FB62F8A2FD539550FBAF
:1067A00063F8F395442D47DE2196452D44DE21966E
:1067B000462D41DE6C96BA9509F0BBCF5F9170FA19
:1067C0007F906F905F904F90FF91EF9178CFFF9304
:1067D000CF93DF936F937F93E42F6091190160FD56
:1067E0001EC0F6EFAA2DBB2DDAE0C49137D0B395C9
:1067F000AA2D96FD33D096FDB395F395AA2DDA9583
:10680000A1F7AA2DAA5F96FDAA5FAA2E7F916F918C
:10681000DF91CF91FF91EF91BF91AF910895F4E88F
:10682000EF77AE2FE2E2EA0FF21DAA0FEA0FF21D98
:10683000AA2DBB2DD6E0C49155D0B395AA2D96FDB7
:1068400051D096FDB395D0FD3196AA2DDA9599F7E2
:10685000AA2DAC5F96FDAC5FAA2ED8CF609138010F
:106860006F936295C7FD629560933801A2D0A3959E
:1068700096FD9FD096FDA395C6FD62956093380165
:1068800098D0A39596FD95D096FDA395C5FD6295EC
:10689000609338018ED0A39596FD8BD096FDA3957D
:1068A000C4FD62956093380184D0A39596FD81D094
:1068B00096FDA395C3FD6295609338017AD0A395A8
:1068C00096FD77D096FDA395C2FD62956093380141
:1068D00070D0A39596FD6DD096FDA3956F916093B2
:1068E0003801089560913801D0FDC295762FC7FF19
:1068F0007295709338015DD0A39596FD5AD096FDA0
:10690000A395762FC6FF72957093380152D0A39548
:1069100096FD4FD096FDA395762FC5FF7295709387
:10692000380147D0A39596FD44D096FDA395762FC8
:10693000C4FF7295709338013CD0A39596FD39D071
:1069400096FDA3956093380108954F93459140308B
:1069500011F44F9108956FDEF9CFFF91EF91EE0F93
:10696000FF1FAF93BF93B591BF3F11F0A5910ED01C
:10697000BF91AF914F934591403031F44F91319792
:10698000F695E7953196099456DEF5CFEF93E091B1
:106990004A01E03021F0EF91AA2EBB2E0895EF912D
:1069A000AE3108F0ADE1B73108F0B6E1AA2EBB2E4A
:1069B0000895CF93DF93C0915001CA1728F0C0917A
:1069C0005101CB1708F003C0DF91CF910895AF9329
:1069D000BF934F935F93C0914A01C53031F0C430EB
:1069E00041F0C37039F0C23008F442C009F465C008
:1069F00082C099C051E0AC3360F5BE3250F5B0FDB5
:106A0000550FB0FD550FA0FD550FB695A695CEE1DB
:106A1000BC9FD1E0C8EDCA0FD21DC00DD11DA2EBA5
:106A2000B2E0CA0FDB1FA881B0913801BE70B295E9
:106A3000A07EBA17A9F0B0913801BE70AB2BAE7E24
:106A4000A883A2EBB2E0CA1BDB0BB881B52BBF70E9
:106A5000B8835F914F91BF91AF91DF91CF9108952E
:106A6000A2EBB2E0CA1BDB0BB8815095B523EFCF88
:106A7000CA2FC770C39540E00894441FCA95E9F730
:106A8000A695A695A695C5E1D0914A01D2FDC0E193
:106A9000BC9FD1E0C8EDCA0FD21DC00DD11DA09181
:106AA0003801A695A17029F44095A881A423A88354
:106AB000D0CFA881A42BA883CCCFCA2F5091380166
:106AC0005695537043E0C37031F0440F440F550F97
:106AD000550FCA95C9F74095A695A695CEE1BC9FDE
:106AE000D1E0C8EDCA0FD21DC00DD11DA881A423CD
:106AF000A52BA883AECFCA2F509138015E704EE00F
:106B0000C17011F4429552954095A695CAE2BC9F7A
:106B1000D1E0C8EDCA0FD21DC00DD11DA881A4239C
:106B2000A52BA88396CF51E0AC33D0F4BE32C0F48D
:106B3000B0FD550FB0FD550FA0FD550FB695A695AC
:106B4000CEE1BC9FD1E0C8EDCA0FD21DC00DD11D52
:106B5000B0913801B27029F0B881B52BBF70B883FD
:106B600078CFB8815095B523F9CFCE3108F0CDE17B
:106B7000EE3108F0EDE1D73108F0D6E1F73108F059
:106B8000F6E1EC1718F40E2EEC2FC02DFD1718F4BB
:106B90000F2EFD2FD02D0895EC1718F40E2EEC2F8C
:106BA000C02DFD1718F40F2EFD2FD02D08950E9433
:106BB00024015F93DADFAC2FBD2FCF93DF93A1D1F8
:106BC000288252EBC50F52E0D51F509138015883EF
:106BD000DF91CF91AE1711F0A395EFCFBF1719F04A
:106BE000AC2FB395EACF5F910C941D010E94240154
:106BF0005F93D2DFAC2FBD2FDCDEA395AE17E1F79C
:106C0000D8DEB395FB17E1F7D4DEAA95AC17E1F710
:106C1000D0DEBA95BD17E1F75F910C941D010E947B
:106C200024015F93B9DFBD2FAC2FC3DEAE1711F087
:106C3000A395FBCFBEDEFB1711F0B395F5CF5F91A7
:106C40000C941D010895B3DF0E9424014F935F93BC
:106C50008CDF4C2FBD2FAC2F54D152EF599351EFF5
:106C6000A395AE1711F05993FBCF53EF5993A42F6F
:106C7000B395BF1739F045D150EF5993AE2F41D19D
:106C80005993F5CFA42F3DD154EF599351EFA395CC
:106C9000AE1711F05993FBCF55EF59935F914F9178
:106CA0000C941D01D0DF5F93AF93BF93CF93DF931D
:106CB000EF93FF935ADFDE0124D15BEF59935CEE33
:106CC000A395AE1711F05993FBCF5CEF5993FF9149
:106CD000EF91DF91CF91CF93DF93EF93FF93DE019D
:106CE000B3950FD15DEF599350E2A395AE1711F014
:106CF0005993FBCF5EEF5993FF91EF91DF91CF91C5
:106D0000CF93DF93EF93FF93DE01B395AF93F9D069
:106D1000A2EBB2E0CA0FDB1F5091380152955E7EA4
:106D20002196AF91A395AE1711F05993FBCFFF9128
:106D3000EF91DF91CF91CF93DF93EF93FF93BD2F2F
:106D4000AC2FBE5FDED05EEE59935DEEA395AE171D
:106D500011F05993FBCF5FEE5993FF91EF91DF91C3
:106D6000CF91BF91AF915F9108950F931F932F9390
:106D70003F93AF93BF93CF93DF93DE010FEFCE1B13
:106D800010F40195C1951FEFDF1B10F41195D195FB
:106D9000CD1760F000C02C2F26950BDEAE1789F0C2
:106DA000A00F2D1BD0F7B10F2C0FF7CF2D2F26954D
:106DB00000DEBF1731F0B10F2C1BD0F7A00F2D0F45
:106DC000F7CFDF91CF91BF91AF913F912F911F915D
:106DD0000F910895AF93A82DA73EE9F3A82DA73EE4
:106DE000E9F7AF910895EF93FF93AF93A093290133
:106DF000FBE8A6FDFCE8F0933B01AF73AA0FFDE8AA
:106E0000E0E8EA0FF21DA591A0932601A591A093B9
:106E10002701209228012092240120922501AF9180
:106E2000FF91EF910895209223014091230140307A
:106E3000E1F3A6C0409122014030E1F708955FD010
:106E4000A2EBCA0FA2E0DA1FA881BA2FAF93A171FB
:106E5000BE7EB295BA2BAF912092230140912301BF
:106E6000403041F440911C014B3110F4A883F6CF1F
:106E7000B883F4CFA88384D042C03F933DED52D075
:106E800020922301409120014470431749F0403083
:106E900021F40E94B007342F03C00E94D607342F7C
:106EA00040912301403061F440911C014B3120F4AA
:106EB00048814F774883E6CF488140684883E2CFD6
:106EC00058815F7758833F910895D1E0C3EECA0F90
:106ED000D21D2092230140912301403061F4409162
:106EE0001C014B3120F448814F774883F4CF48810F
:106EF00040684883F0CF58815F7758830895AA2D62
:106F0000BB2DDEE1BD9FD1E0C8EDCA0FD21DC00D83
:106F1000D11D0895F6DF0F9302EBC00F02E0D01FE2
:106F20000F910895D3E2BD9FD2E0C4E4CA0FD21DF1
:106F3000C00DD11D0895BF93BFEFB1B900001A99DC
:106F4000FECF42B9B4E6BA95F1F72998B4E6BA95FE
:106F5000F1F7299ABF91089545E5E1D00E94823862
:106F6000C8EDD1E0F7E5EEE1BCD0FA95E1F7CF91BD
:106F7000DF91EF91FF914F91442708954F9108952C
:106F80004F934091390141FFF9CF4D7F4093390133
:106F900040914A01463090F7FF93EF93DF93CF93F0
:106FA0004430D1F2403029F44091350147FF13C0FD
:106FB00025C04F9347E4B3D04F914F93405DAFD07E
:106FC0004F91413009F447C0423009F453C0433077
:106FD00009F465C06DC044E50E948F380E94823874
:106FE000C8EDD1E0FEE2EEE17CD0FA95E1F7CF9179
:106FF000DF91EF91FF914F914427089545E40E945E
:107000008F3840914C0163D00E948238C8EDD1E0A6
:10701000F3E0E3E266D00E948238FA95D1F7E3E22A
:10702000F0913A01EF9FC00DD11DF0E1E3E24881FC
:107030004F7742954FD049914F774CD0EA95B9F7A9
:107040000E948238FA9591F7CF91DF91EF91FF91ED
:107050004F91442708954091000139D0409101019A
:1070600036D050D0C8EDD1E0F4E7E5E13AD0FA955A
:10707000E1F7EACF409100012AD04091010127D0E9
:107080004091020124D04091030121D03BD0C8EDB2
:10709000D1E0F4E5EEE125D0FA95E1F7D5CF32D095
:1070A000C8EDD1E0FAE3EAE21CD0FA95E1F7CCCFE3
:1070B000409100010CD04091010109D023D0C8EDCE
:1070C000D1E0F0E4E0E10DD0FA95E1F7BDCF4295D3
:1070D000469547704F70405D4A3308F0495F0C9405
:1070E0008F3848814295F6DF4991F4DFEA95C9F778
:1070F0000C948238BF93B2E0A03009F0B064B4BD04
:10710000BF910895BF934F934DE0B0911801B6FD24
:1071100006D04AE0B7FD03D04F91BF910895BF93C9
:10712000B0913101B030E1F740933201BA95B0939C
:107130003101BF910895BF93B0913301B030E1F7B1
:10714000BA95B0933301B0913301B030E1F740917B
:107150003401BF910895BF93B0913301B030E1F78E
:10716000BA95B0933301409122014D3E41F0B09168
:107170003301B030C1F740913401BF9108954BE124
:10718000BF910895DF93CF93BF93AF93FF93EF9396
:10719000CEE1D7E0ECE0F2E733D0EF91FF91FF933F
:1071A000EF93EEDECCE6D4E0B0912001B2FD7E9606
:1071B00016F026D001C01ED040912201A1E04D3E24
:1071C00069F0A2E0413F51F0A3E0423F39F0A4E072
:1071D000433F21F0A5E0443F09F0DFCFB09120010B
:1071E000B2FDAB5F4A2FEF91FF91AF91BF91CF916D
:1071F000DF910895BEE1A191A993BA95E1F70895B1
:10720000BEE1A591A993BA95E1F708954E4E4E4E71
:107210004E4EC0C0C0C0C0C08080808080802E2EF6
:107220002E2E2E2E6E6E6E6E6E6EDF93CF93BF93EC
:10723000AF93FF93EF93CEE1D7E0ECE0F2E7E0DF2E
:10724000EF91FF91FF93EF93CCE6D4E0D9DFCBCF62
:10725000ACE5B0911801B3FDAFE5ACBDACE5A093D2
:10726000B800A0E0B4FDA1E0A093B9000895FF9399
:10727000EF930F93E0912A01A0912B01B0912C0183
:10728000F0912D010027E2FD0095E5FD0095A4FD9C
:107290000095F7FD0095001FEE1FAA1FBB1FFF1FE3
:1072A000E0932A01A0932B01B0932C01F0932D01C0
:1072B0000F91EF91FF910895DF93CF93BF93AF9319
:1072C000FF93EF934F935F936F937F93A8EDB1E09C
:1072D000C2EBD2E02D922197E9F740E050E012D0C6
:1072E00043954034D9F77F916F915F914F917BCF58
:1072F00067FF05C04F934C2FCD2FD42F4F917C2B80
:10730000660F0895E0E0F6EFF50FE40F6491C09189
:107310003801DC2FD295C07FD07FE3E07727E8DF0C
:107320007295E6DF72957D93EA95C1F753955A30D1
:1073300049F70895DF93CF93BF93AF93FF93EF93F4
:107340004F93A0E8B7E0E0E0F6EFCAE0D0E845915F
:107350004D93DA95E1F7F096F096B096CA95B1F7AD
:107360004F9141CFDF93CF93BF93AF93C0E5D2E06E
:10737000A9E62992AA95E9F7ACEEB4E039922992F0
:107380001197E1F732CFDF93CF93BF93AF93C8ED5F
:10739000D1E0ACE3B0E2009038010CAEB993AA950D
:1073A000E1F723CF0E9424014F935F936F937F9364
:1073B0004F925F926F927F922F9320914A0140905B
:1073C00052015090550160905401709057015091B6
:1073D000530160915601A22FA370E52F660FEE0FA7
:1073E000A33031F0660FEE0FA23011F0660FEE0FF2
:1073F000F62FA0915801A13071F4E20142D0803003
:1074000011F08FE133C0E3013CD0803011F080E215
:107410002DC060D02BC0A23091F4E20132D0803078
:1074200011F08FE123C0E3013BD0803011F082E105
:107430001DC0ACE3BDE06A0E7B1E70D017C0A33048
:1074400011F085E113C0A52DA33010F082E10EC02C
:10745000ACE3BDE04A0E5B1EF20151916191E30184
:1074600010D0803011F080E201C062D02F917F9067
:107470006F905F904F907F916F915F914F910C94BF
:107480001D01CE0F10F48FE10895A0915001CA178D
:10749000D0F7DF0FC0F3B0915101DB17A0F70895CB
:1074A000659FC00DD11D2296D33008F082E108956A
:1074B000A22F5091530160915601E52F660FEE0FF8
:1074C000A33031F0660FEE0FA23011F0660FEE0F11
:1074D000F62F0895571478F0D20134D0E0E9FBE09C
:1074E00064D0D3012FD0E0E9FBE084D053947394AF
:1074F0006A9591F70895560E760E5A947A94D201B1
:1075000021D0E0E9FBE051D0D3011CD0E0E9FBE061
:1075100071D05A947A946A9591F70895F301519332
:107520006193D2010FD041D053946A95D1F7089559
:10753000F20151916191D30105D05CD073946A95A9
:10754000D1F708956F93C8EDD1E0213011F465E1D2
:1075500003C0253069F460E1B69FC00DD11D6A2FCC
:10756000669566956695C60FD21D4A2F6F91089550
:10757000223069F46EE1B69FC00DD11D6A2F669569
:107580006695C60FD21D4A2F440F6F9108956AE287
:10759000B69FC00DD11D6A2F66956695C60FD21D88
:1075A0004A2F440F440F6F9108957F936F93BF93B9
:1075B000AF93652F742F777029F4A991A1936A95E1
:1075C000E1F73FC0B0E8713019F0B6957A95FBCF7E
:1075D0007727A991AB9F703019F0A291A029A193B0
:1075E000119273957617A9F7A991AB9FA291A02943
:1075F000A19327C07F936F93BF93AF93652F742F91
:10760000777029F4A191A9936A95E1F71AC00F93B5
:107610001F930FEF11E0000F110F7A95E1F7652F1F
:107620007881009570230095A191A19F072A099266
:10763000712D6A95C9F768816023672B69930F9153
:107640001F91AF91BF916F917F9108950E94240186
:107650000F931F932F9310E020E0FAE8EE27C091DC
:107660005301CF77D0915601DF7704910C9FA12D64
:10767000E0950491E0950D9FB12DA11729F4B21763
:1076800019F4E39591F724C01A2F2B2FA0915201E2
:10769000B0915501A10FB20F0E94D934A0915201AF
:1076A000B0915501A10FB21B0E94D934A091520193
:1076B000B0915501A11BB21B0E94D934A091520177
:1076C000B0915501A11BB20F0E94D934E39569F620
:1076D0002F911F910F910C941D010E9424010F9373
:1076E0001F932F933F932FEFFAE8EE27C09153019A
:1076F000CF77D0915601DF7704910C9FA12DE095B3
:107700000491E0950D9FB12DB21721F4E395A1F7F7
:107710003F91DECF1A2F2B2FA0915201B09155012E
:107720003A2FB21BA11B310F0E94D934B20FB20FF6
:107730000E94D934B21BB21BA3953A17A8F7E39560
:10774000D9F63F91C5CFFF91EF91EE0FFF1F5BD0B0
:107750003197F695E7953196EF93FF93C8E8D1E01E
:10776000409138014F93FF93EF9361D00E94AD3465
:107770000B0920505245535320454E54455220008A
:10778000EF91FF914F91409338014DDB4A3EE9F76D
:1077900051DB0E94FE1B0895FF91EF91EE0FFF1F3A
:1077A00032D03197F695E7953196EF93FF93C8E87D
:1077B000D1E0409138014F93FF93EF9338D00E946E
:1077C000AD340B08202859296573202F20284E2915
:1077D0006F200000EF91FF914F914093380123DB20
:1077E000493761F0493551F04E3619F04E3409F001
:1077F000F6CF20DB0E94FE1B442708951BDB0E946E
:10780000FE1B41E00895C8E8D1E0459146954F93AD
:10781000477049934F9142954770499358E145917C
:107820004993403011F05A95D1F729920895FF936A
:10783000EF9392E020923601A991B991B295B07779
:10784000A770AB0FAA0FA0933801DF93CF930E94CC
:10785000DC1BC2E0D8E0EBE1FCE00E942336A3E0B1
:10786000B9E00E94C634CF91DF9158E14991403090
:1078700051F0DF93CF935F930E941B335F91CF91C1
:10788000DF915A9599F7409138014295409338011C
:10789000EF91FF9108950E942401C0915201D0916F
:1078A00055010A8119810E3118F4173108F415D0E9
:1078B000A0915401B0915701C0915201D09155014E
:1078C000B983AA83AE3138F4B73128F43CD0737051
:1078D000713009F079D00C941D01C0915201D09102
:1078E00055010A8119812C813B81239F310F2596F7
:1078F000C00DD11DC00DD11D412FE8EDF1E05EE1BD
:10790000549FE00DF11DE00FF21D522F699161931C
:107910005A95E1F74395431781F740914A01463064
:1079200089F0412FEAE8F4E05EE1549FE00DF11D9B
:10793000E00FF21D522F699161935A95E1F743953B
:10794000431781F70895C0915201D09155010A81E2
:1079500019812C813B81239F310F2596C00DD11DAC
:10796000C00DD11D7727412FE8EDF1E05EE1549F76
:10797000E00DF11DE00FF21D522F619169936F70C0
:1079800009F071E05A95C9F74395431769F7E091FB
:107990005201F09155014081742B708340914A014E
:1079A000463089F0412FEAE8F4E05EE1549FE00DB3
:1079B000F11DE00FF21D522F619169935A95E1F785
:1079C0004395431781F70895C0915201D091550115
:1079D0000A8119812C813B81310F2596412FE8EDD9
:1079E000F1E05EE1549FE00DF11DE00FF21D522F1A
:1079F000699161935A95E1F74395431781F7409157
:107A00004A014630C1F0412FEAE8F4E05EE1549FBC
:107A1000E00DF11DE00FF21D522F6991660F28F461
:107A20006E70462E6081607F642961935A95A9F734
:107A30004395431749F708950E9424014F935F939C
:107A40006F93E0913801437001F5A6E1B2E0C4E321
:107A5000D2E0F22D0BD0A0914A01A63031F0A8EC73
:107A6000B4E0C6EED4E0FE2F01D06DC062E15AE171
:107A700049914D935A95E1F7149624966A95B9F772
:107A80005AE1FD935A95E9F708954130E9F4ACE4E1
:107A9000B4E0CBE4D4E0F22D0BD0A0914A01A430A5
:107AA00031F0AEEFB6E0CDEFD6E0FE2F01D04BC007
:107AB00063E159E14A914E935A95E1F7FE93149789
:107AC00025976A95B1F70895423001F5ACE4B4E02A
:107AD000CEE2D4E0F22D0BD0A0914A01A43031F0D7
:107AE000AEEFB6E0C0EED6E0FE2F01D02CC062E1D2
:107AF0005AE14A914E935A95E1F7149724976A9563
:107B0000B9F75AE1FE935A95E9F70895A6E1B2E074
:107B1000C7E1D2E0F22D0BD0A0914A01A43031F0A0
:107B2000A8ECB4E0C9ECD4E0FE2F01D00CC063E1B6
:107B300059E149914D935A95E1F7FD932596149695
:107B40006A95B1F708956F915F914F910C941D0163
:107B50004F935F937F93FFDA4B3111F481E015C0AF
:107B60004130C9F7E8DA642FE6DA4095641711F07E
:107B700088E20BC070E85527DEDA540F49937A95F6
:107B8000D9F7D9DA451729F488277F915F914F916A
:107B9000089589E2FACF4F935F937F9341E0BFDA74
:107BA000462FBDDA4095BBDA70E855274991540F4E
:107BB000B6DA7A95D9F7452FB2DA7F915F914F9176
:107BC00008955E984CE54093B80044E84093BC00AB
:107BD00044E94093BC00089544EA0EC05093BB00B2
:107BE00044E80AC044EC08D05091BB00089544E832
:107BF00003D05091BB0008954093BC004091BC005D
:107C000047FFFCCF6091B900687F0895E5DF6830D9
:107C100089F4572F550F5E70506AE0DF683151F4D8
:107C20005B2FDCDF683231F45A2FD8DF683211F471
:107C3000882708958FE05F915F91CACFE7DFCCDF9F
:107C4000603169F4572F550F5E70516AC7DF603499
:107C500031F4CDDF683519F411968827B9CF8FE05C
:107C6000B7CF052ED3DF502DB9DF683219F4119646
:107C70008827AECF8FE00895AFDF6830A9F4572F83
:107C80005770550F5169AADF603471F4ABDF60356E
:107C900059F4A52FACDF683539F4BB27550FAA1F5F
:107CA00008F4B095882794CF8FE092CF8827D830FA
:107CB00020F082E24F914F914FEF0895F7DFF9994D
:107CC000FECFD2BDC1BDF89A40B521960895EEDF32
:107CD0008827F999FDCFD2BDC1BDF89A40B44416AA
:107CE00011F42196089540BDF894FA9AF99A78947F
:107CF000F999FECFF89A21960895AF93DFDF41936B
:107D0000AA95E1F7AF910895AF934191E0DFAA956D
:107D1000E1F7AF9108954EBD4DB547FFFDCF4EB58C
:107D2000089588272C9847EDF6DF4427F4DF2C9A36
:107D30004C7B4432B1F34C31A1F38827443A19F01B
:107D40004C3909F081E108958827EBDF803021F07C
:107D500040E040939C1008954C3911F448E0F9CF6D
:107D600040E1F7CFF1DF403009F40895440F440FAC
:107D7000440F440F4A950895AA0FBB1F4B2FCBDF2A
:107D80004A2FC9DF422DC7DFB695A79508958030E9
:107D900059F44F93C6DF803031F42C9845E5BBDFB2
:107DA000EBDF2C9ABEDF4F910895803059F44F934A
:107DB000B8DF803031F42C9843E5ADDFDDDF2C9A5D
:107DC000B0DF4F910895803051F44F93AADF803097
:107DD00029F42C9846E89FDFCFDF2C9A4F91089525
:107DE0001196B0939D10A0939E101197ECCF2DD2B9
:107DF000CEDF48D0E8CF7F93772710D07F910895CA
:107E00007F9371E00BD0D42F72E008D0C42F7F9104
:107E100008957F9373E002D07F910895803099F4A4
:107E200080DF803081F42C9842ED75DFAA0FBB1FF4
:107E3000A3954B2F70DF4A2F6EDF472F6CDFB6956F
:107E4000A79502D02C9A089566DF65DF64DF63DFB3
:107E500062CF8030B1F465DF803099F42C9842ED28
:107E60005ADFAA0FBB1F4B2F56DF4A2F54DF472F75
:107E7000440F51DFB695A795E7DFD42F4CDFC42F11
:107E80002C9A08957F9370E010D07F9108957F938E
:107E900071E04D2F0AD072E04C2FC0DF7F91089522
:107EA0007F9373E0BBDF7F9108958030A1F44F93FF
:107EB00038DF4F91803079F42C984F9347E82BDFCF
:107EC000442729DF41E027DF472F25DF4F914F93DC
:107ED00022DF2C9A4F910895803091F422DF803078
:107EE000D1F72C984F9347E816DF442714DF40E082
:107EF00012DF472F10DF4F914F930DDF2C9A4F91D8
:107F000008958030D1F4DF93CF934F935F9309DFCF
:107F1000803079F42C9847E8FEDE4427FCDE4427C5
:107F2000FADE40E0F8DE55274991F5DE5A95E1F793
:107F30002C9A5F914F91CF91DF9108958030B1F4E9
:107F40004F935F93EEDE803079F42C9847E8E3DEC0
:107F50004427E1DE4427DFDE40E0DDDE55274FEF3A
:107F6000DADE5A95E1F72C9A5F914F9108958030AF
:107F7000E1F4DF93CF934F935F93D3DE803089F4A6
:107F80002C9846EDC8DE4427C6DE4427C4DE40E018
:107F9000C2DE4427C0DE5527BEDE49935A95E1F77D
:107FA0002C9A5F914F91CF91DF910895BF93AF933A
:107FB000DF93CF934F935F937F93C6DE403001F4FE
:107FC000BDDF4FE05FDF44276BDFAA27BB27FBDE67
:107FD00011964DEFCA2FCF70C13009F44CEF52DF2C
:107FE00044275EDFCC27DD2752DFEDDE1196A0307F
:107FF00019F445EE0E941B3340919C10B41749F7C9
:108000000AC0BF93AF93DF93CF934F935F937F9358
:108010009BDE403091F47F915F914F91CF91DF9142
:10802000AF91BF910895B42FAA271197F2DEC42F04
:10803000BB27AA27EEDE4C1731F4A9DEEADE439512
:108040002FDFC1DEE8CF1196E4DE4C17E1F7F5CF64
:10805000DF93CF934F939BDE4DEFCA2FCF70C1308C
:1080600009F44CEF0FDFCCDE219611DF67DFABDECA
:108070004F91CF91DF910895FF93EF93DF93CF93CB
:10808000BF93AF93AA27BB27ED015EDE4030A1F07E
:10809000F42FB1DE4C3F41F04D3F31F04B3A21F02F
:1080A0004F3018F0403908F421961196BF1789F720
:1080B0004427DF1709F441E06FC00F93BF93AF93DC
:1080C0004F93AA27BB27ED01FD013EDE403099F01A
:1080D000042F91DE4D3F49F4DF93CF9391DE4D2F76
:1080E000CF91DF914F3F21F021964C3F09F431961B
:1080F0001196B01771F74F91AF91BF910F910895FD
:10810000FF93EF93DF93CF934F932F931DDE403078
:10811000A9F0AA27BB276FDE242FB0919D10A09154
:108120009E1040911401B41710F0A2E0BB27FD018E
:1081300062DE4D3F31F464DED21718F42F914F9177
:108140002DC0159640919C10B41709F4BB27BF179A
:1081500079F7AE1769F7AA27BB2719DE4CDE4F3F28
:1081600031F0405F242F8EDE2EDEDF01E1CFAFEF56
:10817000BFEFE4CFFF93EF93DF93CF93BF93AF9322
:108180004F935F936F937F93DFDD403061F481E124
:108190007F916F915F914F91AF91BF91CF91DF919F
:1081A000EF91FF91089551D0B41710F08BE1F0CF0B
:1081B00022DE4C3F11F087E1EBCF40916A01403065
:1081C00011F48BE1E5CF413810F08BE1E1CF75DFA1
:1081D000D03021F4C41710F488E1DACFC0E9DBE035
:1081E00050E06FEF69935A95E9F7A8DE1196B093C6
:1081F0009D10A0939E1040916A01C0E9DBE04F936F
:108200007FDFB993A9934BEA3DDEDF93CF93F8DD8F
:1082100021963DDECF91DF91FCDD42DEE1DDF1DE36
:108220004F914A9561F711D0C0E9DBE06ADE4091D9
:108230006C0128DEDF93CF93E3DD219628DECF911A
:10824000DF91E7DD2DDEBFDDA3CFA0916801A29510
:10825000BA2FA07FBF70119608950E9424014F93FA
:108260005F937F937727F1DFC6DD4C3F69F0F1DD47
:10827000DF3F49F0BF93AF93DE01EADEAF91BF91DC
:10828000C0DE7F5FA1F7E4DE7F915F914F910C9498
:108290001D010E9424014F935F937F932F93AA2780
:1082A000BB273FDDA8DD242FD0DFA5DD4C3F39F40F
:1082B00089E12F917F915F914F910C941D017091F5
:1082C0006A01703810F08BE1F4CFC3DDDF3F11F4A9
:1082D0008BE1EFCFDE01CCE3DDE040916C0141307A
:1082E00009F4D395423009F4DE5F0BDEDF93CF93C0
:1082F00087DDD21759F02196CADDCF91DF917BDD62
:10830000C1DD87DDCDDD5FDD7CDED3CFA1DEF8DE34
:1083100077DD2196BCDDCF91DF914BEAB3DD79DDCE
:10832000BFDD51DDED0191DF32DD70916A01770F24
:108330004D2FD2DD73954C2FCFDD5DDDA3DD69DDE3
:10834000AFDD41DDB6CF0E9424014F935F937F9351
:108350007CDF51DD4C3F31F48EE17F915F914F9195
:108360000C941D0170916A01703810F08BE1F5CF0B
:1083700070DDDF3F11F48BE1F0CFDE0108DDCCE3EF
:10838000DDE040916C01413009F4D395423009F4AD
:10839000DE5FEDDDE2CF0E9424014F935F937F9378
:1083A00054DF29DD4C3F11F48EE1D7CF772751DD23
:1083B000DE0170E0E8E8F1E04CDDD193C193739504
:1083C0007032D1F7CACF0004080D11161A1F2328E6
:1083D0002C3035393D42464A4F53575B5F64686CD9
:1083E0007074787C7F83878B8F92969A9DA1A4A7C7
:1083F000ABAEB1B5B8BBBEC1C4C6C9CCCFD1D4D663
:10840000D9DBDDDFE2E4E6E8E9EBEDEEF0F2F3F4F0
:10841000F6F7F8F9FAFBFCFCFDFEFEFFFFFFFFFF9D
:10842000FFFF000000CCC000333000FFF000000C64
:10843000CCCCCCCC333CCCFFFCCC000333CCC33312
:10844000333333FFF333000FFFCCCFFF333FFFFF56
:10845000FFFFA5A5A506FF600000000000000000CA
:10846000000000000000000000000000000000000C
:108470000000000000000EAE000004E000AAE800CA
:10848000EE4E000000444040AA000066FF666842CD
:10849000C4A248A000000044000048884042224096
:1084A0000A4A0004E40000048000E00000004022CA
:1084B0004880EAAAE04C44E0E2E8E0E2E2E0AAE236
:1084C00020E8E2E0E8EAE0E24880EAEAE0EAE2E026
:1084D0000404000404802484200E0E00842480C23E
:1084E00068E400EEE04AAEA0CACAC0688860CAAAC2
:1084F000C0E8C8E0E8C88068EA60AAEAA0E444E00E
:10850000E22A60AC8CA08888E0AEAAA0CAAAA04AE1
:10851000AA40EAE8804AAA60EAECA068E2C0E44423
:1085200040AAAAE0AAAA40AAAEA0AA4AA0AA444089
:10853000E248E064446004A400C444C04A0000006F
:1085400000E04400004AAEA0CACAC0688860CAAA57
:10855000C0E8C8E0E8C88068EA60AAEAA0E444E0AD
:10856000E22A60AC8CA08888E0AEAAA0CAAAA04A81
:10857000AA40EAE8804AAA60EAECA068E2C0E444C3
:1085800040AAAAE0AAAA40AAAEA0AA4AA0AA444029
:10859000E248E024C4204444448464808842208C1F
:0285A000EC806D
:1086000000F900F5F3F1F2FC00FAF8F6F4EB5E0085
:10861000F7000000007131000000797361773200CB
:108620000063786465343300002076667472350028
:10863000006E6268677A360000006D6A7537380030
:10864000002C6B696F303900002E2D6C00707E009D
:1086500000000000002700000000EA2B00230000BB
:10866000003C00000000EC00003100343700000046
:10867000302C32353638ED00FB2B332D2A390000F3
:1086800000F900F5F3F1F2FC00FAF8F6F4EB000063
:10869000F70000000051210000005953415722000B
:1086A00000435844452440000020564654522500BB
:1086B000004E4248475A260000004D4A552F2800D8
:1086C000003B4B494F3D2900003A5F4C00503F00B2
:1086D00000000000006000000000EA2A00270000FF
:1086E000003E00000000EC000031003437000000C4
:1086F00030E932353638ED00FB2B332D2A390000B6
:108700000000000000000000000000000000000069
:108710000000000000000000000000000000000059
:108720000000000000000000000000000000000049
:1087300000000000000000C000000000000000C1B8
:10874000000000000000000000002F0000000000FA
:1087500000000000000000000000EA000000C2006D
:10876000000000000000000000E100E2E000000066
:10877000E8E9E500E3E4ED00FB2BE72D2AE6000045
:1087800000000000000000000000000000000000E9
:108790000000000000400000000000000000000099
:1087A00000000000000000000000000000000000C9
:1087B000000000000000000000000000007B5B00E3
:1087C00000000000007D5D000000000000007E0051
:1087D00000000000000000000000005C000000003D
:1087E000007C00000000000000E100E2E00000006A
:1087F000EFEEE500E3E4ED00FB2BE72D2AE60000B9
:1088000000F900F5F3F1F2FC00FAF8F6F4EB5E0083
:10881000F70000000071310000007A7361773200C8
:108820000063786465343300002076667472350026
:10883000006E62686779360000006D6A753738002F
:10884000002C6B696F303900002E2F6C3B702D00AF
:10885000000027005B3D00000000EA5D007E000094
:10886000000000000000EC00003100343700000080
:10887000302C32353638ED00FB2B332D2A390000F1
:1088800000F900F5F3F1F2FC00FAF8F6F4EB000061
:10889000F70000000051210000005A5341574000EA
:1088A00000435844452423000020564654522500D6
:1088B000004E424847595E0000004D4A55262A00A6
:1088C000003C4B494F292800003E3F4C3A505F0086
:1088D000000022007B2B00000000EA7D007C0000ED
:1088E000000000000000EC00003100343700000000
:1088F00030E932353638ED00FB2B332D2A390000B4
:108900000000000000000000000000000000000067
:108910000000000000000000000000000000000057
:108920000000000000000000000000000000000047
:1089300000000000000000C000000000000000C1B6
:10894000000000000000000000002F0000000000F8
:1089500000000000000000000000EA000000C2006B
:10896000000000000000000000E100E2E000000064
:10897000E8E9E500E3E4ED00FB2BE72D2AE6000043
:1089800000000000000000000000000000000000E7
:1089900000000000000000000000000000000000D7
:1089A00000000000000000000000000000000000C7
:1089B00000000000000000000000000000000000B7
:1089C00000000000000000000000000000000000A7
:1089D0000000000000000000000000000000000097
:1089E000000000000000000000E100E2E0000000E4
:1089F000EFEEE500E3E4ED00FB2BE72D2AE60000B7
:108A0000FFFFFFFFFFFFFFFFFFFFFFFEFEFEFEFE7B
:108A1000FEFEFDFDFDFDFDFCFCFCFCFBFBFBFBFA93
:108A2000FAFAF9F9F9F8F8F8F7F7F6F6F6F5F5F4D1
:108A3000F4F3F3F2F2F2F1F0F0EFEFEEEEEDEDEC35
:108A4000EBEBEAEAE9E8E8E7E6E6E5E4E4E3E2E1BD
:108A5000E1E0DFDEDEDDDCDBDADAD9D8D7D6D5D46B
:108A6000D4D3D2D1D0CFCECDCCCBCAC9C9C8C7C63A
:108A7000C5C4C3C2C1BFBEBDBCBBBAB9B8B7B6B529
:108A8000B4B2B1B0AFAEADACAAA9A8A7A6A5A3A237
:108A9000A1A09E9D9C9B99989796949392918F8E5E
:108AA0008D8B8A898786858382817F7E7D7B7A789C
:108AB0007776747371706F6D6C6A696766656362EF
:108AC000605F5D5C5A595756545351504E4D4B4A56
:108AD0004847454442413F3E3C3B393836353332C6
:108AE000302E2D2B2A2827252422201F1D1C1A1941
:108AF00017161412110F0E0C0B09070604030100C0
:108B00000C11161A1E2225282B2D2F313233333407
:108B100034343434343434343535363738393B3CF6
:108B20003E40434547494B4D4F5152535454545482
:108B3000545351504E4C4A4745423F3D3A383634E3
:108B40003231302F2E2E2E2F303132333536383A07
:108B50003C3E4042444647494A4B4D4E4E4F505092
:108B60005050505050504F4E4D4C4B494846434149
:108B70003E3B37332F2B27221D18130D0802FDF81B
:108B8000F3EEE9E5E1DDDAD7D4D2D0CECDCCCCCB53
:108B9000CBCBCBCBCBCBCBCBCACAC9C8C7C6C4C344
:108BA000C1BFBCBAB8B6B4B2B0AEADACABABABAB98
:108BB000ABACAEAFB1B3B5B8BABDC0C2C5C7C9CB17
:108BC000CDCECFD0D1D1D1D0CFCECDCCCAC9C7C5D3
:108BD000C3C1BFBDBBB9B8B6B5B4B2B1B1B0AFAF28
:108BE000AFAFAFAFAFAFB0B1B2B3B4B6B7B9BCBE51
:108BF000C1C4C8CCD0D4D8DDE2E7ECF2F7FD02075F
:108C0000000A141D272F383F464B505457595959C5
:108C1000585654504C48433E39332E2925201C19B0
:108C200016141211111112131517191C1F222527C2
:108C30002A2C2E303132323232312F2D2B28252260
:108C40001F1C191613110F0D0C0B0A0A0A0B0C0E20
:108C500010121416181A1C1E1F2020201F1E1C196B
:108C600016120D0803FDF7F0EAE3DDD6D1CBC6C23C
:108C7000BFBDBBBABBBCBEC2C6CBD1D7DFE6EFF728
:108C80000008101920282E34393D41434445444200
:108C9000403D39342E29221C150F0802FCF7F2ED55
:108CA000E9E6E3E1E0DFDFDFE0E1E3E5E7E9EBED83
:108CB000EFF1F3F4F5F5F5F4F3F2F0EEECE9E6E3B9
:108CC000E0DDDAD7D4D2D0CECDCDCDCDCECFD1D37D
:108CD000D5D8DADDE0E3E6E8EAECEDEEEEEEEDEB3A
:108CE000E9E6E3DFDAD6D1CCC6C1BCB7B3AFABA9F6
:108CF000A7A6A6A6A8ABAFB4B9C0C7D0D8E2EBF57B
:108D000080675342352B221C16120E0C09070605EC
:108D1000040000000000000000000000000000004F
:108D2000807E7B79777572706E6C6A686664636149
:108D30005F5D5C5A5857555352504F4D4C4B494804
:108D40004745444341403F3E3D3C3B39383736354B
:108D50003433323231302F2E2D2C2B2B2A29282838
:108D60002726252524232322222120201F1F1E1DE4
:108D70001D1C1C1B1B1A1A19191818181717160076
:108D8000890091009A00A300AD00B700C200CE0098
:108D9000DA00E700F4000301120123013401460167
:108DA0005A016E0184019B01B301CD01E901060264
:108DB0002502450268028C02B302DC020803360376
:108DC00067039B03D2030C0449048B04D0041905E8
:108DD0006705B90510066C06CE063507A307170808
:108DE000930815099F09320ACD0A720B200CD80C82
:108DF0009C0D6B0E460F2F1025112A123F13641481
:108E0000F894A0E02A2EA1E03A2EA0E1AEBFAFEF89
:108E1000ADBFB0E0A0E0AA95F1F7BA95D9F7AAEBFB
:108E2000A4B9AFEFA5B9A0E8A7B9A0E0A8B9A0EF91
:108E3000AAB9AFEFABB9A6B1AF71A09335014B9909
:108E40005DC0B2ECB0938000B9E1B0938100F4E072
:108E5000A2FFF4E0F0938700FEEFA2FFF6EFF0939D
:108E6000860020928900FAE5F0938800A2E0A093A2
:108E70006F00A0E4A4BDA1E0A5BDA1E3A7BD209221
:108E8000C000A0E1A093C100A6E6A093C200E0EA62
:108E9000FFE87ED0A2E2B591B993AA95E1F705B7B4
:108EA000036005BF0E7F05BF7894A8EC68D0B09131
:108EB000C600B83719F0AA95C9F720C0E0ECFFE862
:108EC00067D045E140D0C8EDD1E020D046E03BD0AE
:108ED000E0E0F0E0CCE3DFE019D046E034D0CCEBCA
:108EE000DFE014D0FE3820F40E9476793296789430
:108EF00046E029D0AEEEB1E01BD0ECCFF89405B738
:108F0000016005BF0C7F05BF0C94000028D04430E1
:108F100039F446E018D0B0913101B030E1F7EECF2E
:108F200050E81DD01CD01BD049935A95E1F717C0CB
:108F30004F2F429501D04F2F4F70405D4A3308F0BC
:108F4000495F4D930895BF93B0913101B030E1F77F
:108F500040933201BA95B0933101BF910895BF9308
:108F6000B0913301B030E1F7BA95B0933301B091CD
:108F70003301B030E1F740913401BF910895AF93D0
:108F8000A82DA73EE9F3A82DA73EE9F7AF910895D4
:108F9000C8EDD1E0A2E2B591B993AA95E1F70895A1
:108FA0004156522D436869704261736963322028CB
:108FB0004631313D557064617465205379732920C1
:108FC000426F6F746C6F61646572204572726F726C
:108FD000202845534320746F206578697429202028
:0E900000202020202020202020202020FFFFE4
:0E9C0000202020202020202020202020FFFFD8
:0EA80000202020202020202020202020FFFFCC
:0EB40000202020202020202020202020FFFFC0
:0EC00000202020202020202020202020FFFFB4
:0ECC0000202020202020202020202020FFFFA8
:0ED80000202020202020202020202020FFFF9C
:0EE4000048656C6C6F20576F726C64204EFF85
:10E410000E94670000EC0E9456000E9473000000FA
:10E4200048656C6C6F20576F726C642100000EE0C1
:10E430000E9456000E947300020070726573732080
:0CE4400071000E947B004137E1F7089555
:10F000000C9400474F934091840040918500433019
:10F01000D1F740918400409185004030D1F70DC078
:10F0200000000000000000000000000000000000E0
:10F03000000000000C941C784F935F936F93FF9334
:10F04000EF93DF93CF93BF93AF930F921F92FFB7CE
:10F05000FF93C4E1D1E0B9A5B7FF5C98B7FD5C9A16
:10F060004B99BE7F4B9BB160B9A7830C921CE9A161
:10F07000F92DF03029F4F82DFA3010F1F63EF8F0C1
:10F08000FCE0E2FFFDEE8F1639F45E98E3FF17C057
:10F09000B2E8B093800013C0F1E1E2FFF3EF8F1606
:10F0A00039F45E9AE3FF0BC0B2ECB093800007C066
:10F0B000F9E3E2FFF7E08F1611F4882499242EC0BB
:10F0C0003E9933C0A0918400A63ED0F3A73E00F045
:10F0D000A83E00F0A93E00F0AA3E00F0A8EDB1E085
:10F0E000F6EFF80DC0E2ED91549140E060E848B9C8
:10F0F000ED9156FD66B90000000055FD66B904901B
:10F1000054FD66B9CA95000053FD66B900000000C1
:10F1100052FD66B9502D59F7000028B816D0E0917D
:10F12000C600E63711F40C947E47FF91FFBF1F9095
:10F130000F90AF91BF91CF91DF91EF91FF916F91C0
:10F140005F914F913E9B18950895A0913D01E091EC
:10F150003301E03091F0EF3F21F4A0FD0EC0EEE36B
:10F160000CC0EA95F5EFB491B5FF07C0B09134013A
:10F17000B695A0FBB7F9B0933401E0933301E09169
:10F180003101E03091F0EF3F19F4E0E5AF770DC0C9
:10F19000EA95F5EFB491B4FF08C0B0913201B0FB2D
:10F1A0000894B795A7F9B0933201E0933101A09389
:10F1B0003D010895A0913D01E0913301E03091F0CF
:10F1C000EF3F21F4A0FD0EC0ECE70CC0EA95F5EF8F
:10F1D000B491B7FF07C0B0913401B695A0FBB7F961
:10F1E000B0933401E0933301E0913101E030E9F272
:10F1F000EF3F19F4E0E9AF77D8CFEA95F5EFB49196
:10F20000B6FFD3CFB0913201B0FB0894B795A7F900
:10F21000B0933201CACF40911801C8EFD7E00E94E5
:10F22000673E409165010E94673E0895C8EFD7E0B0
:10F230000E945E3E409318010E945E3E409365012D
:10F240000895FF93EF93DF93CF93AF9300D1E093B3
:10F250004001F0934101AF91CF91DF91EF91FF9188
:10F260000895E0914001F0914101A0E2A99FE00DD5
:10F27000F11DB096C0EBD1E0A0E2B591B993AA958B
:10F28000E1F7BFEFB993089547B740FDFDCFB7BF92
:10F29000E8950E94027847B740FDFBCF089547B735
:10F2A00040FDFDCFB7BFE89547B740FDFDCF0895BE
:10F2B00047B746FF0895B1E1E7DFFACFF8944E2F44
:10F2C000407E19F4B3E0E0DFF3DFA0E1099019908C
:10F2D000B1E0E5DF3296AA95C9F7E03009F008956C
:10F2E0003297B5E0D1DFE4DF32960895F8944F937A
:10F2F000BF93AF93B3E0C8DFDBDF3297CCE3DFE04F
:10F30000A0E8329609901990B1E0C9DFAA95C9F733
:10F31000B5E0BADFCDDFAF91BF914F910895E09195
:10F320004001F0914101B097ACE0B591B993AA9535
:10F33000E1F7A0913501A7FD0895A6EAB2E0CA0F52
:10F34000DB1FACE0B0913801B993AA95E9F70895B5
:10F35000E0E0F0E9A0E0BCE0492F403029F3EA0FFB
:10F36000FB1F4A95FACF409149014770AF93ECE0FB
:10F37000F0E9ACE0A49FF00D4491EC50AF910895FA
:10F38000F89463D0C0EBD1E0A3EEB1E05CE04D9126
:10F3900049935A95E1F742E4499353E140E2B99326
:10F3A0005A95E9F7A0978ADF9927B3E2B99FA4E4B9
:10F3B000B2E0A00DB11DC8E8D1E050E24D914993F3
:10F3C0005A95E1F7299250E24A91403219F4288285
:10F3D0005A95D1F70E944D1AC0EBD1E06FDF93959B
:10F3E0009F3519F77894089530D0A3EEB1E05CE032
:10F3F00045914D935A95E1F77496992750E2A0EB09
:10F40000B1E045914D935A95E1F7A8E8B1E040E2AB
:10F4100053E24D935A95E9F7FF93EF939F930E9420
:10F420002E1B9F91EF91FF91C8E8D1E0B3E2B99F05
:10F43000A1E4B2E0A00DB11D53E249914D935A955C
:10F44000E1F793959F35D1F6089540914901AF9327
:10F45000BF93E0E0F0E947704295A0ECA49FE00D77
:10F46000F11DBF91AF910895CCE3DFE04CE050E295
:10F4700059934A95E9F75FEF599343E150E2599365
:10F480004A95E9F740EF5FEF59934A95E9F7DDDFD9
:10F490002DDF3296CCE3DFE040E25FEF59934A95EF
:10F4A000E9F74BE04F9322DF32964F914A95D1F71F
:10F4B00078940895472F4770CADFFF93EF93C5DF15
:10F4C000AF91BF914CE04F93CCE3DFE040E055912A
:10F4D00059934A95E1F7FF93EF93FD0107DF3296C9
:10F4E000DF01EF91FF914F914A9569F77894089564
:10F50000010101010101210101010101012181012B
:10F510000100002100110101010121D101010101BE
:10F520002101110101010121D1010101012101117B
:10F530000101010121D101010101010111010101BB
:10F540000101D1010101010101110101010101C10B
:10F55000010101010101010101000101C1010101DC
:10F56000010101010101010001C1010101010100CD
:10F57000010101010101410001010101010101003D
:10F58000000000400000000000000000000000003B
:10F59000000000000000000000000000000000006B
:10F5A000000000000000000000000000000000005B
:10F5B000000000000000000000000000000000004B
:10F5C000000000000000000000000000000000003B
:10F5D000000000000000000000000000000000002B
:10F5E000100000000000000000000000000000000B
:10F5F00020000000000000000000000000000000EB
:10F60000009010800090108000901080009010807A
:10F61000FC28288004C0145028282800000000007E
:10F6200000000000000000000000000000000000DA
:10F6300000000000000000000000000000000000CA
:10F6400000000000000000000000000000000000BA
:10F6500000000000000000000000000000000000AA
:10F66000000000000000000000000000000000009A
:10F67000000000000000000000000000000000008A
:10F6800028C004C00000000000000000000000804E
:10F69000C0A0888400000000000000002088FCB4A6
:10F6A0000028000008A08080000004C028800024FA
:10F6B00028008000000044288000C004C418000016
:10F6C00000282828280028281818280000000000F2
:10F6D0008090808008A084408080C8A400004C8472
:10F6E00000000000000000008080601800802828D2
:10F6F000280000002828002828282800002CE8904E
:10F700000090108000901080009010800090108079
:10F710007C444480A8A814504844440024000000BD
:10F7200000183C3C185028280C3000000000000055
:10F73000241824400C401440242400000C003024E1
:10F7400024244424444040246424106460646424D9
:10F7500044244424406464646464404800481800BD
:10F76000300060000400140060180C6028000000E5
:10F7700000000000300000000000000C18306000A5
:10F7800028A004C0808044283C3C3C000044A88061
:10F79000C0A08884000000000000008040847C58E5
:10F7A000182800001090808004C004C028FC287C29
:10F7B00028440C00000044EC8000C004C424000075
:10F7C00000282828286C2828C01828640000000079
:10F7D0008088A41010908440C004C8A400008C80CD
:10F7E000287C008080004084FCF8303000002448F1
:10F7F000280000002828002828282800002CE8C01D
:10F800000090108000901080009010800090108078
:10F81000FC44448080801450444444283C00000050
:10F8200000183C3C20546C181818181800000004EC
:10F830006428640C14603064646428281800186418
:10F84000646464646460606464180C6C605864642C
:10F8500064646464186464646464046000183C0054
:10F860001800600004003400600000601800000010
:10F870000000000030000000000000181818601898
:10F88000449008A0C4C4806C0000001C1844A880E8
:10F89000C0A0888400000000000080804084FCB488
:10F8A0002428282820888080A4A00C60448044401C
:10F8B00028440C40844444800000C0046C2400446C
:10F8C00000282828286C8080C018445440844810A0
:10F8D0008084BCB020888820D834C8A440848C8020
:10F8E0002C7C00C4C4448080C0082830008020885C
:10F8F000280000002828002828282800002CE8A03C
:10F900000090108000901080009010800090108077
:10F910007C808080808010908480804424186424BF
:10F9200000183C40780C7830300C7C180000000C3B
:10F93000681804183C44600C6464282830400C04A7
:10F94000046464606460606064180C78607C546473
:10F9500064646460186464643C640C60301864001F
:10F960000C2444242C2430207428146C185C742437
:10F970004824742448646464646440181818300C83
:10F9800044881090C4BC446C24246434286C6C807B
:10F99000C0A08884000000000080808080807CEC13
:10F9A000404444442088408490A00C6044FC286477
:10F9B00080440C40844444280000C0046C2400802F
:10F9C00028444444446C80806018C44C600C18186F
:10F9D0008080BC1040848820E82CC8A480804C849F
:10F9E000EC2400C4EC448080C008144800802088C7
:10F9F000280000002828002828282800002CE8E4F7
:10FA00000090108000901080009010800090108076
:10FA1000FC808080B098109080ECEC44003C6464E2
:10FA20000018003C24183000300C2440004000181E
:10FA30007C180C0C6C044418242000006000040C9A
:10FA40002C6444606444447040180C50607C7C64B6
:10FA50004464442418646464183C18607C180000F2
:10FA6000000464606864486454180C78187C54641A
:10FA70006C6C5460306464643C640C30180C188006
:10FA800080841090C4F8806C04646440406C6C8086
:10FA9000C0A0888400000000808080808080FCB44A
:10FAA0001880442840844084808418308080282432
:10FAB00000440C40844444440000C00428241880BE
:10FAC0008080844080A800006018C480A008402482
:10FAD000A4B0BC4080808080E82CC8A488104084FA
:10FAE000E42428C4EC44D480C00814848080208896
:10FAF000288020882088808020888020882CE8F03A
:10FB00000000000090909090101010108080808075
:10FB10007C8080801090B098408080440040646475
:10FB2000001800401C307800300C7C182800003091
:10FB300054181804400464186404282830400C1831
:10FB40007C4064606460606464180C78606468641D
:10FB5000607C780418643C7C3C1830600C18000011
:10FB6000002064606440306464180C50187C646445
:10FB70006C6C602430646464182C181818180C0C11
:10FB800080842088C4C444C420646430286C6C80A1
:10FB9000C0A08884000000008080808080807CEC91
:10FBA00018008044408440848080301880FC801895
:10FBB00044448040844444440000C0042800244459
:10FBC0008080844080A800443018C480A00824406D
:10FBD000BCD0A41084404084E82CC8A44C8480800D
:10FBE000482428C4EC44F880C0081484808020880D
:10FBF000288020882088808020888020882CE82801
:10FC00000000000090909090101010108080808074
:10FC1000FC8080801090808084C4A8440000643CF4
:10FC20000000003C44686C00181818181800286080
:10FC3000641830640C646430640C281818001800D0
:10FC40007C6464646460606464186C6C60646464A4
:10FC500060686C6418643C7C641860600018000084
:10FC6000006464646460302064180C781864646410
:10FC7000482460043C683C7C3C0830181818041880
:10FC800044882088C4C4808064646818186C6C80C0
:10FC9000C0A0888400000080808080808080FCB4C8
:10FCA000400080804084208880843018DC80284098
:10FCB00000446040844444280000C0046C0024C414
:10FCC00044444444446C80443018C44C600C1818BC
:10FCD000BCB0808084402088E44CC4C44C848080C4
:10FCE000282400C4EC44D4D0FCF8148480002828D4
:10FCF000280028280000280028282820882CE83000
:10FD00000000000090909090101010108080808073
:10FD10007C4480441450808044EC442800004458C3
:10FD20000018003C18082C000C300000300028009F
:10FD3000242440240C242430242800300C003018C3
:10FD4000246444244440602464242864406464247B
:10FD5000602C64241824182464184048004800408B
:10FD6000002044242424300464246C6C246464241F
:10FD7000600C6044182C183C6404400C18300400DB
:10FD8000449040848080442820242C0000A8448093
:10FD9000C0A08884000080808080808040847C585F
:10FDA000240080288080208890A0600CDCFC44180F
:10FDB00028446040844444EC0000C0046C002400EB
:10FDC00028002828286C804418184454408410487F
:10FDD000BCB0808080801090D094C0048C8040841F
:10FDE000284000C4C444FCF880802884800028286F
:10FDF000280028280000280028282820882CE830FF
:10FE00000000000090909090101010108080808072
:10FE1000FC4480441450A8A84080440000006000C6
:10FE200000000000000000000000000000000000D2
:10FE300000000000000000000000000000000000C2
:10FE400000000000000000000000000000000000B2
:10FE500000000000000000000000000000000000A2
:10FE60000000000000000024000028000000000046
:10FE700060080000000000000024000000000000F6
:10FE800028A08080000000000000000000A844803E
:10FE9000C0A0888400808080808080804084FCECCA
:10FEA0001800444480801090A4A0C004DC806C3C06
:10FEB00000446000004400800080C004C4002400AE
:10FEC00028002828286C282818182864000000001A
:10FED000A4B08080844008A0C8A480808C800000EA
:10FEE000444000808000D4F8408430480000282836
:10FEF000280028280000280028282824482CE8006A
:10FF00000000000090909090101010108080808071
:10FF10007C2880281450109080EC28000000C0003D
:10FF200000000000000000000000000000000000D1
:10FF300000000000000000000000000000000000C1
:10FF400000000000000000000000000000000000B1
:10FF500000000000000000000000000000000000A1
:10FF60000000000000000000000000000000000091
:10FF70000000000000000000000000000000000081
:10FF800028C0808000000000000000000000008009
:10FF9000C0A08884808080808080808020887C5879
:10FFA00000004480808008A004C0C0048CFCA858D5
:10FFB00000006000004400280080C004C40000006D
:10FFC00028002828280028281818280000000000E9
:10FFD0008080000084400000C8A400004824000085
:10FFE00000000000000080800000600080002828E1
:10FFF000280028280000280028282828282CE80085
:00000001FF
